:020000040000FA
:0408000039EF08F0D4
:1008100003B213EF05F0F2B42EEF05F09EB036EF01
:1008200005F09EB23EEF05F0F2A81AEF04F0F2B226
:1008300025EF04F0F2A620EF04F0F2B022EF04F06E
:10084000E8EF07F0F296F290FF00CD90F2929EA0B2
:100850002FEF04F00101533F2FEF04F0542BAEC1F2
:10086000B2F1AFC1B3F1B0C1B4F1B1C1B5F1AAC138
:10087000AEF1ABC1AFF1ACC1B0F1ADC1B1F1A6C148
:10088000AAF1A7C1ABF1A8C1ACF1A9C1ADF1A2C158
:10089000A6F1A3C1A7F1A4C1A8F1A5C1A9F19EC168
:1008A000A2F19FC1A3F1A0C1A4F1A1C1A5F19AC178
:1008B0009EF19BC19FF19CC1A0F19DC1A1F196C188
:1008C0009AF197C19BF198C19CF199C19DF1CECF4E
:1008D00096F1CFCF97F153C198F154C199F1CF6AF6
:1008E000CE6A0101536B546B9E90CD800FBC0F8E6E
:1008F0000FBA7EEF04F00F8AE8EF07F00F8C0FBEFF
:10090000BAEF04F096C19AF197C19BF198C19CF19E
:1009100099C19DF19AC19EF19BC19FF19CC1A0F12B
:100920009DC1A1F19EC1A2F19FC1A3F1A0C1A4F1FB
:10093000A1C1A5F1A2C1A6F1A3C1A7F1A4C1A8F1CB
:10094000A5C1A9F1A6C1AAF1A7C1ABF1A8C1ACF19B
:10095000A9C1ADF1AAC1AEF1ABC1AFF1ACC1B0F16B
:10096000ADC1B1F1AEC1B2F1AFC1B3F1B0C1B4F13B
:10097000B1C1B5F101015E6B5F6B606B616B96514C
:100980005E2797515F2398516023995161239A51B3
:100990005E279B515F239C5160239D5161239E5193
:1009A0005E279F515F23A0516023A1516123A25173
:1009B0005E27A3515F23A4516023A5516123A65153
:1009C0005E27A7515F23A8516023A9516123AA5133
:1009D0005E27AB515F23AC516023AD516123AE5113
:1009E0005E27AF515F23B0516023B1516123B251F3
:1009F0005E27B3515F23B4516023B5516123D89072
:100A00000101613360335F335E33D890010161339C
:100A100060335F335E33D8900101613360335F33FD
:100A20005E33E8EF07F00392030103EE00F080511C
:100A30007F0BE92604C0EFFF802B8151805D700B96
:100A4000D8A48B8200008051815D700BD8A48B925A
:100A500081518019D8B40790E8EF07F0F2940101B2
:100A6000453FE8EF07F0462BE8EF07F09E900101C5
:100A7000533FE8EF07F0542BE8EF07F09E92040095
:100A800062A143EF05F007B495EF05F007B095EFCD
:100A900005F01EC620F61FC621F61CC61EF61DC692
:100AA0001FF61AC61CF61BC61DF606C608F607C6B4
:100AB00009F604C606F605C607F602C604F603C61E
:100AC00005F626C628F627C629F624C626F625C624
:100AD00027F622C624F623C625F60EC610F60FC644
:100AE00011F60CC60EF60DC60FF60AC60CF60BC6AE
:100AF0000DF62EC630F62FC631F62CC62EF62DC6B4
:100B00002FF62AC62CF62BC62DF616C618F617C6D3
:100B100019F614C616F615C617F612C614F613C63D
:100B200015F620EC2AF0B8EC29F0077C07ACB0EF02
:100B300005F0C274C2B4AAEF05F0C3CFB3F5C4CFB9
:100B4000B4F50501D890B433B333D890B433B3338C
:100B5000B1EF05F0C3CF55F1C4CF56F1B1EF05F0B9
:100B6000C28207B41EEF06F047C14BF148C14CF1F9
:100B700049C14DF14AC14EF15EC162F15FC163F1FD
:100B800060C164F161C165F196C1B6F197C1B7F179
:100B900098C1B8F199C1B9F19AC1BAF19BC1BBF141
:100BA0009CC1BCF19DC1BDF19EC1BEF19FC1BFF111
:100BB000A0C1C0F1A1C1C1F1A2C1C2F1A3C1C3F1E1
:100BC000A4C1C4F1A5C1C5F1A6C1C6F1A7C1C7F1B1
:100BD000A8C1C8F1A9C1C9F1AAC1CAF1ABC1CBF181
:100BE000ACC1CCF1ADC1CDF1AEC1CEF1AFC1CFF151
:100BF000B0C1D0F1B1C1D1F1B2C1D2F1B3C1D3F121
:100C0000B4C1D4F1B5C1D5F1B3C5B5F5B4C5B6F528
:100C1000B5C5B7F5B6C5B8F5010155515B275651B5
:100C20005C23E86A5D230E2E1EEF06F05CC157F1CF
:100C30005DC158F15B6B5C6B5D6B078E0201002F31
:100C4000E8EF07F03C0E006F00C10CF101C10DF19F
:100C500002C10EF103C10FF104C110F105C111F180
:100C600006C112F107C113F108C114F109C115F150
:100C70000AC116F10BC117F134C135F105012F512D
:100C8000000AD8B4E7EF06F005012F51010AD8B4E5
:100C900071EF06F005012F51020AD8B4B2EF06F049
:100CA00005012F51030AD8B4B2EF06F005012F5108
:100CB000040AD8B4B2EF06F005012F51050AD8B4E2
:100CC000B2EF06F005012F51060AD8B4B2EF06F0D4
:100CD00005012F51070AD8B4B2EF06F02F6BE7EFEA
:100CE00006F0050153677CEF06F054677CEF06F0D1
:100CF00055677CEF06F0566780EF06F0E7EF06F0E9
:100D000057C500F158C501F159C502F15AC503F1A3
:100D10000101010E046F000E056F000E066F000E3C
:100D2000076F29EC28F000C157F501C158F502C141
:100D300059F503C15AF50067A5EF06F00167A5EF65
:100D400006F00267A5EF06F00367E7EF06F053C56C
:100D500057F554C558F555C559F556C55AF50F8878
:100D6000E7EF06F005013067B8EF06F0E7EF06F0B1
:100D70000FBECDEF06F010A0D2EF06F001014767DD
:100D8000C9EF06F04867C9EF06F04967C9EF06F0FA
:100D90004A67CDEF06F0D2EF06F007AED2EF06F0CD
:100DA000E4EF06F00501312FE7EF06F03C0E316F5E
:100DB000302FE7EF06F00101000E626FE00E636F67
:100DC000A50E646F010E656F0501306B0F8805017C
:100DD000626B33B7EDEF06F062810CC100F10DC11B
:100DE00001F10EC102F10FC103F110C104F111C1F3
:100DF00005F112C106F113C107F114C108F115C1C3
:100E000009F116C10AF117C10BF135C134F100C166
:100E10000CF101C10DF102C10EF103C10FF104C1CA
:100E200010F105C111F106C112F107C113F108C19A
:100E300014F109C115F10AC116F10BC117F134C142
:100E400035F101018A672CEF07F08B672CEF07F073
:100E50008C672CEF07F08D6730EF07F060EF07F03D
:100E60008EC100F18FC101F190C102F191C103F176
:100E70000101010E046F000E056F000E066F000EDB
:100E8000076F29EC28F000C18EF101C18FF102C17A
:100E900090F103C191F1006755EF07F0016755EF3D
:100EA00007F0026755EF07F0036760EF07F08AC1AC
:100EB0008EF18BC18FF18CC190F18DC191F10F80BA
:100EC000D57ED5BE69D0D6CF47F1D7CF48F145C141
:100ED00049F1E86AE8CF4AF1109047C100F148C1F2
:100EE00001F149C102F14AC103F101010A0E046F87
:100EF000000E056F000E066F000E076F29EC28F03C
:100F000003AF1080010154A792EF07F00F9A0F9CD6
:100F10000F9E0101000E5E6F600E5F6F3D0E606FF1
:100F2000080E616F010147BFA2EF07F04867A2EF0B
:100F300007F04967A2EF07F04A67A2EF07F0F288CF
:100F4000C7EF07F0F2985E6B5F6B606B616B966B3F
:100F5000976B986B996B9A6B9B6B9C6B9D6B9E6B65
:100F60009F6BA06BA16BA26BA36BA46BA56BA66B15
:100F7000A76BA86BA96BAA6BAB6BAC6BAD6BAE6BC5
:100F8000AF6BB06BB16BB26BB36BB46BB56BD76A55
:100F9000D66A0101456B466B0CC100F10DC101F130
:100FA0000EC102F10FC103F110C104F111C105F12D
:100FB00012C106F113C107F114C108F115C109F1FD
:100FC00016C10AF117C10BF135C134F1E8EF07F092
:100FD00002C0E0FF005001C0D8FF1000A6B2EEEF43
:100FE00007F00CC0A9FF0BC0A8FFA69EA69CA68474
:100FF000F29E550EA76EAA0EA76EA682F28EA6943A
:10100000A6B200EF08F00C2A1200A96EA69EA69CBC
:10101000A680A8500C2A120004012C0E826FFBEC53
:101020000AF024EC29F00C5005EC08F0E8CF00F1B0
:101030000C5005EC08F0E8CF01F101AF25EF08F006
:101040000101FF0E026FFF0E036FC7EC28F0296746
:1010500031EF08F00401200E826FFBEC0AF036EF4E
:1010600008F004012D0E826FFBEC0AF0F1EC26F083
:101070001200076A0F6A106A0F010D0EC16E860E0C
:10108000C06E030EC26E0F01680E896E130E926E53
:10109000080E8A6E8A6AF30E936E8B6A900E946EB7
:1010A000F18EF19E0E6A01015B6B5C6B5D6B576BA1
:1010B000586BF29A0101476B486B496B4A6B4B6B5B
:1010C0004C6B4D6B4E6B4F6B506B516B526B456B5A
:1010D000466BD76AD66A0F01280ED56EF28A9D90AC
:1010E000B00ECD6E01015E6B5F6B606B616B626B0E
:1010F000636B646B656B666B676B686B696B536B7B
:10110000546BCF6ACE6A0F9A0F9C0F9E9D80760E0D
:10111000CA6E9D8202013C0E006FCC6A160E05EC71
:1011200008F0E8CF00F1170E05EC08F0E8CF01F168
:10113000180E05EC08F0E8CF02F1190E05EC08F0E6
:10114000E8CF03F1010103AFC0EF08F024EC29F070
:10115000160E0C6E00C10BF0EEEC07F0170E0C6EC5
:1011600001C10BF0EEEC07F0180E0C6E02C10BF093
:10117000EEEC07F0190E0C6E03C10BF0EEEC07F06D
:1011800000C18AF101C18BF102C18CF103C18DF163
:1011900000C18EF101C18FF102C190F103C191F143
:1011A0001A0E05EC08F0E8CF00F11B0E05EC08F074
:1011B000E8CF01F11C0E05EC08F0E8CF02F11D0E9E
:1011C00005EC08F0E8CF03F1010103AF16EF09F0D9
:1011D00024EC29F01A0E0C6E00C10BF0EEEC07F0B7
:1011E0001B0E0C6E01C10BF0EEEC07F01C0E0C6E2A
:1011F00002C10BF0EEEC07F01D0E0C6E03C10BF0FC
:10120000EEEC07F01A0E05EC08F0E8CF00F11B0E2B
:1012100005EC08F0E8CF01F11C0E05EC08F0E8CF72
:1012200002F11D0E05EC08F0E8CF03F100C192F1C8
:1012300001C193F102C194F103C195F1240EAC6E8A
:10124000900EAB6E240EAC6E080EB86E000EB06E33
:101250001F0EAF6E0401806B816B0F01900EAB6EA1
:101260000F019D8A0301806B816BC26B8B92B3EC83
:101270002FF0B3EC2FF0E9EC32F094EC2DF0200ECF
:1012800005EC08F0E8CF2FF505012F51FF0AD8A48F
:1012900051EF09F02F6B200E0C6E2FC50BF0EEEC0A
:1012A00007F00501010E306F3C0E316F250E05EC85
:1012B00008F0E8CF00F1260E05EC08F0E8CF01F1C8
:1012C000270E05EC08F0E8CF02F1280E05EC08F037
:1012D000E8CF03F1010103AF88EF09F024EC29F016
:1012E000250E0C6E00C10BF0EEEC07F0260E0C6E16
:1012F00001C10BF0EEEC07F0270E0C6E02C10BF0F3
:10130000EEEC07F0280E0C6E03C10BF0EEEC07F0CC
:1013100000C153F501C154F502C155F503C156F59D
:1013200000C157F501C158F502C159F503C15AF57D
:10133000290E05EC08F0E8CF5BF505015C515B5D1B
:10134000D8A05BC55CF505012F51020A0EE181B8FA
:10135000B5EF09F005015C2FB2EF09F05BC55CF554
:10136000B5EF09F081BA28EF33F0210E05EC08F053
:10137000E8CF00F1220E05EC08F0E8CF01F1230ED2
:1013800005EC08F0E8CF02F1240E05EC08F0E8CFF8
:1013900003F1010103AFFBEF09F024EC29F0210E6A
:1013A0000C6E00C10BF0EEEC07F0220E0C6E01C1CA
:1013B0000BF0EEEC07F0230E0C6E02C10BF0EEEC1E
:1013C00007F0240E0C6E03C10BF0EEEC07F0210EBB
:1013D00005EC08F0E8CF00F1220E05EC08F0E8CFAC
:1013E00001F1230E05EC08F0E8CF02F1240E05EC24
:1013F00008F0E8CF03F100C15DF501C15EF502C15F
:101400005FF503C160F5CBEC2CF08DEC2BF0DDEC3F
:101410002AF005012F51030A12E005012F51040A99
:101420001DE005012F51050A24E005012F51060A90
:1014300032E005012F51070A38E05EEF0AF0ACC533
:1014400000F101010F0E001701010051000A36E002
:1014500001010051050A32E05BEF0AF0ACC500F172
:1014600001010F0E001701010051000A27E05BEF98
:101470000AF00501AC51000A21E00501AC51150A42
:101480001DE00501AC51300A19E00501AC51450AD7
:1014900015E05BEF0AF00501AC51000A0FE0050111
:1014A000AC51300A0BE05BEF0AF00501AC51000AC9
:1014B00005E05BEF0AF081BA28EF33F088EC2AF000
:1014C00007900001F28EF28C07B085EF24F00FB088
:1014D00066EF1FF00FB82AEF19F003018051811950
:1014E0007F0BD8B485EF24F013EE00F081517F0B11
:1014F000E126812BE7CFE8FFE00BD8B485EF24F09D
:1015000023EE82F0C2513F0BD926E7CFDFFFC22B7B
:10151000DF50780AD8A485EF24F007808EC100F14F
:101520008FC101F190C102F191C103F10101040EDB
:10153000046F000E056F000E066F000E076F29EC9A
:1015400028F000AFADEF0AF00101030E8E6F000E20
:101550008F6F000E906F000E916F03018251720A1F
:10156000D8B466EF1FF08251520AD8B466EF1FF06C
:101570008251750AD8B466EF1FF08251630AD8B45D
:1015800041EF21F08251690AD8B421EF1CF0825159
:101590007A0AD8B434EF1DF08251490AD8B4C0EFAA
:1015A0001BF08251500AD8B4DEEF1AF08251700A53
:1015B000D8B421EF1BF08251540AD8B44CEF1BF081
:1015C0008251740AD8B492EF1BF08251730AD8B4D6
:1015D00096EF1EF08251530AD8B4FBEF1EF08251F1
:1015E0004C0AD8B48CEF11F08251760AD8B40FEFC0
:1015F0000BF076EF21F0040114EE00F080517F0B28
:10160000E12682C4E7FF802B120004010D0E826FD9
:10161000FBEC0AF00A0E826FFBEC0AF012000301E9
:101620008351300AD8B45DEF0CF003018351310AC5
:10163000D8B494EF0CF003018351320AD8B449EFC7
:101640000EF003018351330AD8B4FEEF0FF003010B
:101650008351340AD8B4A4EF10F003018351730A04
:10166000D8B43CEF0BF003018351760AD8B43EEFB7
:101670000BF0D8A476EF21F03CEC0BF00401760ED1
:10168000826FFBEC0AF00401760E826FFBEC0AF02D
:1016900004012C0E826FFBEC0AF0A1EC25F0040192
:1016A0002C0E826FFBEC0AF00101036B026B3BC650
:1016B00001F13AC600F101AF63EF0BF00101FF0E3B
:1016C000026FFF0E036FC7EC28F029676AEF0BF07B
:1016D0006FEF0BF004012D0E826FFBEC0AF02FC1AF
:1016E00082F40401300E8227FBEC0AF030C182F450
:1016F0000401300E8227FBEC0AF031C182F40401B0
:10170000300E8227FBEC0AF032C182F40401300E65
:101710008227FBEC0AF033C182F40401300E8227E9
:10172000FBEC0AF004012C0E826FFBEC0AF00101C5
:10173000036B026B3DC601F13CC600F101AFA6EFA1
:101740000BF00101FF0E026FFF0E036FC7EC28F0D4
:101750002967ADEF0BF0B2EF0BF004012D0E826F95
:10176000FBEC0AF02FC182F40401300E8227FBEC5F
:101770000AF030C182F40401300E8227FBEC0AF03B
:1017800031C182F40401300E8227FBEC0AF032C131
:1017900082F40401300E8227FBEC0AF033C182F49C
:1017A0000401300E8227FBEC0AF004012C0E826F3C
:1017B000FBEC0AF00101036B026B3FC601F13EC670
:1017C00000F101AFE9EF0BF00101FF0E026FFF0E18
:1017D000036FC7EC28F02967F0EF0BF0F5EF0BF083
:1017E00004012D0E826FFBEC0AF02FC182F404017C
:1017F000300E8227FBEC0AF030C182F40401300E77
:101800008227FBEC0AF031C182F40401300E8227FA
:10181000FBEC0AF032C182F40401300E8227FBECAB
:101820000AF033C182F40401300E8227FBEC0AF087
:1018300004012C0E826FFBEC0AF00101036B026BBA
:1018400037C601F136C600F101AF2CEF0CF00101F3
:10185000FF0E026FFF0E036FC7EC28F0296733EF0E
:101860000CF038EF0CF004012D0E826FFBEC0AF047
:101870002FC182F40401300E8227FBEC0AF030C144
:1018800082F40401300E8227FBEC0AF031C182F4AD
:101890000401300E8227FBEC0AF032C182F404010D
:1018A000300E8227FBEC0AF033C182F40401300EC3
:1018B0008227FBEC0AF08BEF19F00401760E826FA1
:1018C000FBEC0AF00401300E826FFBEC0AF004011D
:1018D0002C0E826FFBEC0AF092EC29F024EC29F03C
:1018E00000C600F101C601F1C7EC28F030C182F456
:1018F0000401300E8227FBEC0AF031C182F40401AE
:10190000300E8227FBEC0AF032C182F40401300E63
:101910008227FBEC0AF033C182F40401300E8227E7
:10192000FBEC0AF08BEF19F00401760E826FFBECF2
:101930000AF00401310E826FFBEC0AF0078401010A
:10194000036B026B02C600F103C601F101AFADEFFC
:101950000CF0FF0E026FFF0E036F0101076B066BA9
:1019600004C604F105C605F105AFBBEF0CF0FF0E90
:10197000066FFF0E076F2EEC28F00101076B066B58
:1019800006C604F107C605F105AFCBEF0CF0FF0E5C
:10199000066FFF0E076F2EEC28F00101076B066B38
:1019A00008C604F109C605F105AFDBEF0CF0FF0E28
:1019B000066FFF0E076F2EEC28F0D890010103335D
:1019C000023301330033D890010103330233013372
:1019D000003304012C0E826FFBEC0AF00101036B53
:1019E000026B01C101F100C100F101AFFDEF0CF08C
:1019F0000101FF0E026FFF0E036FC7EC28F029678D
:101A000004EF0DF009EF0DF004012D0E826FFBECD9
:101A10000AF02FC182F40401300E8227FBEC0AF099
:101A200030C182F40401300E8227FBEC0AF031C190
:101A300082F40401300E8227FBEC0AF032C182F4FA
:101A40000401300E8227FBEC0AF033C182F404015A
:101A5000300E8227FBEC0AF00101036B026B0AC611
:101A600000F10BC601F101AF3AEF0DF0FF0E026F6E
:101A7000FF0E036F0101076B066B0CC604F10DC668
:101A800005F105AF48EF0DF0FF0E066FFF0E076F73
:101A90002EEC28F00101076B066B0EC604F10FC691
:101AA00005F105AF58EF0DF0FF0E066FFF0E076F43
:101AB0002EEC28F00101076B066B10C604F111C66D
:101AC00005F105AF68EF0DF0FF0E066FFF0E076F13
:101AD0002EEC28F0D8900101033302330133003398
:101AE000D8900101033302330133003304012C0E7B
:101AF000826FFBEC0AF00101036B026B01C101F183
:101B000000C100F101AF8AEF0DF00101FF0E026F7D
:101B1000FF0E036FC7EC28F0296791EF0DF096EFE9
:101B20000DF004012D0E826FFBEC0AF02FC182F440
:101B30000401300E8227FBEC0AF030C182F404016C
:101B4000300E8227FBEC0AF031C182F40401300E22
:101B50008227FBEC0AF032C182F40401300E8227A6
:101B6000FBEC0AF033C182F40401300E8227FBEC57
:101B70000AF00101036B026B12C600F113C601F1FA
:101B800001AFC7EF0DF0FF0E026FFF0E036F0101F3
:101B9000076B066B14C604F115C605F105AFD5EF4A
:101BA0000DF0FF0E066FFF0E076F2EEC28F00101FF
:101BB000076B066B16C604F117C605F105AFE5EF16
:101BC0000DF0FF0E066FFF0E076F2EEC28F00101DF
:101BD000076B066B18C604F119C605F105AFF5EFE2
:101BE0000DF0FF0E066FFF0E076F2EEC28F0D89059
:101BF00001010333023301330033D8900101033371
:101C000002330133003304012C0E826FFBEC0AF027
:101C10000101036B026B01C101F100C100F101AFD1
:101C200017EF0EF00101FF0E026FFF0E036FC7ECFE
:101C300028F029671EEF0EF023EF0EF004012D0EA1
:101C4000826FFBEC0AF02FC182F40401300E822770
:101C5000FBEC0AF030C182F40401300E8227FBEC69
:101C60000AF031C182F40401300E8227FBEC0AF045
:101C700032C182F40401300E8227FBEC0AF033C13A
:101C800082F40401300E8227FBEC0AF007948BEFFC
:101C900019F00401760E826FFBEC0AF00401320E9B
:101CA000826FFBEC0AF007840101036B026B1AC61A
:101CB00000F11BC601F101AF62EF0EF0FF0E026FE3
:101CC000FF0E036F0101076B066B1CC604F11DC6F6
:101CD00005F105AF70EF0EF0FF0E066FFF0E076FF8
:101CE0002EEC28F00101076B066B1EC604F11FC61F
:101CF00005F105AF80EF0EF0FF0E066FFF0E076FC8
:101D00002EEC28F00101076B066B20C604F121C6FA
:101D100005F105AF90EF0EF0FF0E066FFF0E076F97
:101D20002EEC28F0D8900101033302330133003345
:101D3000D8900101033302330133003304012C0E28
:101D4000826FFBEC0AF00101036B026B01C101F130
:101D500000C100F101AFB2EF0EF00101FF0E026F02
:101D6000FF0E036FC7EC28F02967B9EF0EF0BEEF46
:101D70000EF004012D0E826FFBEC0AF02FC182F4ED
:101D80000401300E8227FBEC0AF030C182F404011A
:101D9000300E8227FBEC0AF031C182F40401300ED0
:101DA0008227FBEC0AF032C182F40401300E822754
:101DB000FBEC0AF033C182F40401300E8227FBEC05
:101DC0000AF00101036B026B22C600F123C601F188
:101DD00001AFEFEF0EF0FF0E026FFF0E036F010178
:101DE000076B066B24C604F125C605F105AFFDEFB0
:101DF0000EF0FF0E066FFF0E076F2EEC28F00101AC
:101E0000076B066B26C604F127C605F105AF0DEF7B
:101E10000FF0FF0E066FFF0E076F2EEC28F001018A
:101E2000076B066B28C604F129C605F105AF1DEF47
:101E30000FF0FF0E066FFF0E076F2EEC28F0D89004
:101E400001010333023301330033D890010103331E
:101E500002330133003304012C0E826FFBEC0AF0D5
:101E60000101036B026B01C101F100C100F101AF7F
:101E70003FEF0FF00101FF0E026FFF0E036FC7EC83
:101E800028F0296746EF0FF04BEF0FF004012D0EFD
:101E9000826FFBEC0AF02FC182F40401300E82271E
:101EA000FBEC0AF030C182F40401300E8227FBEC17
:101EB0000AF031C182F40401300E8227FBEC0AF0F3
:101EC00032C182F40401300E8227FBEC0AF033C1E8
:101ED00082F40401300E8227FBEC0AF00101036B4F
:101EE000026B2AC600F12BC601F101AF7CEF0FF0A7
:101EF000FF0E026FFF0E036F0101076B066B2CC60E
:101F000004F12DC605F105AF8AEF0FF0FF0E066F45
:101F1000FF0E076F2EEC28F00101076B066B2EC633
:101F200004F12FC605F105AF9AEF0FF0FF0E066F13
:101F3000FF0E076F2EEC28F00101076B066B30C611
:101F400004F131C605F105AFAAEF0FF0FF0E066FE1
:101F5000FF0E076F2EEC28F0D890010103330233F7
:101F600001330033D89001010333023301330033CE
:101F700004012C0E826FFBEC0AF00101036B026B73
:101F800001C101F100C100F101AFCCEF0FF001017F
:101F9000FF0E026FFF0E036FC7EC28F02967D3EF27
:101FA0000FF0D8EF0FF004012D0E826FFBEC0AF05A
:101FB0002FC182F40401300E8227FBEC0AF030C1FD
:101FC00082F40401300E8227FBEC0AF031C182F466
:101FD0000401300E8227FBEC0AF032C182F40401C6
:101FE000300E8227FBEC0AF033C182F40401300E7C
:101FF0008227FBEC0AF007948BEF19F00401760EB0
:10200000826FFBEC0AF00401330E826FFBEC0AF0E6
:1020100004012C0E826FFBEC0AF085C382F4FBEC0A
:102020000AF0640E0D6E03018551320A02E16A0E58
:102030000D6E03018551330A02E1700E0D6E03012E
:102040008551340A02E1760E0D6E03018551350A81
:1020500002E17C0E0D6E03018551360A02E1820E0B
:102060000D6E03018651780A65E00DC00CF065EC39
:1020700029F02981030187512D0AD8B442EF10F0CD
:102080000101299188C32FF189C330F18AC331F14D
:102090008BC332F18CC333F172EC29F0E9EC28F0F8
:1020A00000C10BF0EEEC07F001C10BF0EEEC07F015
:1020B00065EC29F0298103018E512D0AD8B463EF14
:1020C00010F0010129918FC32FF190C330F191C31A
:1020D00031F192C332F193C333F172EC29F0E9ECA0
:1020E00028F000C10BF0EEEC07F001C10BF0EEECB4
:1020F00007F065EC29F02981030195512D0AD8B428
:1021000084EF10F00101299196C32FF197C330F1AC
:1021100098C331F199C332F19AC333F172EC29F0CB
:10212000E9EC28F000C10BF0EEEC07F001C10BF078
:10213000EEEC07F00DC00CF00CEC08F00CEC08F025
:102140000CEC08F08BEF19F00401760E826FFBECBB
:102150000AF00401340E826FFBEC0AF00301845193
:10216000780AD8B47CEF11F03E0E0C6E65EC29F0C5
:102170002981030185512D0AD8B4C1EF10F0010166
:10218000299186C32FF187C330F188C331F189C308
:1021900032F18AC333F172EC29F0E9EC28F000C186
:1021A0000BF0EEEC07F001C10BF0EEEC07F065EC84
:1021B00029F0298103018C512D0AD8B4E2EF10F0E7
:1021C000010129918DC32FF18EC330F18FC331F1FD
:1021D00090C332F191C333F172EC29F0E9EC28F0AD
:1021E00000C10BF0EEEC07F001C10BF0EEEC07F0D4
:1021F00065EC29F02981030193512D0AD8B403EF2E
:1022000011F00101299194C32FF195C330F196C3C8
:1022100031F197C332F198C333F172EC29F0E9EC54
:1022200028F000C10BF0EEEC07F001C10BF0EEEC72
:1022300007F065EC29F0298103019A512D0AD8B4E1
:1022400024EF11F0010129919BC32FF19CC330F1C0
:102250009DC331F19EC332F19FC333F172EC29F07B
:10226000E9EC28F000C10BF0EEEC07F001C10BF037
:10227000EEEC07F065EC29F029810301A1512D0A4C
:10228000D8B445EF11F001012991A2C32FF1A3C3E6
:1022900030F1A4C331F1A5C332F1A6C333F172EC1E
:1022A00029F0E9EC28F000C10BF0EEEC07F001C1D9
:1022B0000BF0EEEC07F065EC29F029810301A85141
:1022C0002D0AD8B466EF11F001012991A9C32FF1AD
:1022D000AAC330F1ABC331F1ACC332F1ADC333F1BA
:1022E00072EC29F0E9EC28F000C10BF0EEEC07F0FD
:1022F00001C10BF0EEEC07F03E0E0C6E0CEC08F09A
:102300000CEC08F00CEC08F00CEC08F00CEC08F00D
:102310000CEC08F08BEF19F003018351300AD8B4AC
:102320004DEF14F003018351310AD8B45BEF15F07F
:1023300003018351320AD8B4C9EF15F00301835168
:10234000330AD8B4D9EF15F003018351340AD8B455
:10235000E9EF15F003018351350AD8B42FEF19F0D6
:1023600003018351360AD8B45DEF19F0030183519C
:10237000460AD8B483EF18F0030183514D0AD8B44C
:10238000C6EF12F0030183516D0AD8B4E0EF12F0EA
:10239000030183515A0AD8B4D5EF14F003018351D5
:1023A000490AD8B45DEF1AF003018351500AD8B43A
:1023B0008FEF19F003018351540AD8B408EF1AF0D3
:1023C00003018351630AD8B400EF13F00301835172
:1023D000430AD8B4F8EF13F003018351730AD8B459
:1023E000FEEF12F003018351610AD8B413EF12F02B
:1023F00003018351650AD8B49DEF14F003018351A2
:10240000450AD8B4ABEF14F003018351620AD8B483
:10241000B9EF14F003018351420AD8B4C7EF14F0A6
:10242000D8A476EF21F004014C0E826FFBEC0AF089
:102430000401610E826FFBEC0AF08DEC2BF00401BD
:102440002C0E826FFBEC0AF024EC29F0ABC500F1F6
:102450000101C7EC28F031C182F40401300E82275B
:10246000FBEC0AF032C182F40401300E8227FBEC4F
:102470000AF033C182F40401300E8227FBEC0AF02B
:1024800004012C0E826FFBEC0AF024EC29F0ACC5A1
:1024900000F10101C7EC28F031C182F40401300ED3
:1024A0008227FBEC0AF032C182F40401300E82274D
:1024B000FBEC0AF033C182F40401300E8227FBECFE
:1024C0000AF004012C0E826FFBEC0AF024EC29F0D8
:1024D000ADC500F10101C7EC28F031C182F404015F
:1024E000300E8227FBEC0AF032C182F40401300E78
:1024F0008227FBEC0AF033C182F40401300E8227FC
:10250000FBEC0AF004012C0E826FFBEC0AF024ECC9
:1025100029F0AEC500F10101C7EC28F031C182F409
:102520000401300E8227FBEC0AF032C182F4040170
:10253000300E8227FBEC0AF033C182F40401300E26
:102540008227FBEC0AF004012C0E826FFBEC0AF0F0
:1025500024EC29F0B3C500F10101C7EC28F031C12A
:1025600082F40401300E8227FBEC0AF032C182F4BF
:102570000401300E8227FBEC0AF033C182F404011F
:10258000300E8227FBEC0AF08BEF19F065EC29F096
:1025900084C333F172EC29F0E9EC28F0200E0C6EC4
:1025A00000C10BF0EEEC07F000C12FF505012F5133
:1025B000000A06E005012F51010A02E033EC2CF07D
:1025C00004014C0E826FFBEC0AF004014D0E826F89
:1025D000FBEC0AF004012C0E826FFBEC0AF024ECF9
:1025E00029F02FC500F1C7EC28F033C182F40401B3
:1025F000300E8227FBEC0AF08BEF19F028EF33F056
:1026000004014C0E826FFBEC0AF00401630E826F32
:10261000FBEC0AF0DDEC2AF004012C0E826FFBECDF
:102620000AF015EC13F08BEF19F024EC29F0B1C58A
:1026300000F10101003B0F0E0017C7EC28F033C179
:1026400082F40401300E8227FBEC0AF0B1C500F1E0
:1026500001010F0E01010017C7EC28F033C182F40D
:102660000401300E8227FBEC0AF004012D0E826F6C
:10267000FBEC0AF0B0C500F10101003B0F0E0017A2
:10268000C7EC28F033C182F40401300E8227FBEC42
:102690000AF0B0C500F101010F0E01010017C7ECEF
:1026A00028F033C182F40401300E8227FBEC0AF0DB
:1026B00004012D0E826FFBEC0AF0AFC500F10101A1
:1026C000003B0F0E0017C7EC28F033C182F4040161
:1026D000300E8227FBEC0AF0AFC500F101010F0EAE
:1026E00001010017C7EC28F033C182F40401300E59
:1026F0008227FBEC0AF00401200E826FFBEC0AF04B
:10270000AEC500F10F0E01010017C7EC28F033C170
:1027100082F40401300E8227FBEC0AF00401200E43
:10272000826FFBEC0AF0ADC500F101010101003B35
:102730000F0E0017C7EC28F033C182F40401300EED
:102740008227FBEC0AF0ADC500F101010F0E01017B
:102750000017C7EC28F033C182F40401300E822741
:10276000FBEC0AF004013A0E826FFBEC0AF0ACC5F8
:1027700000F10101003B0F0E0017C7EC28F033C138
:1027800082F40401300E8227FBEC0AF0ACC500F1A4
:1027900001010F0E01010017C7EC28F033C182F4CC
:1027A0000401300E8227FBEC0AF004013A0E826F1E
:1027B000FBEC0AF0ABC500F10101003B0F0E001766
:1027C000C7EC28F033C182F40401300E8227FBEC01
:1027D0000AF0ABC500F101010F0E0017C7EC28F09D
:1027E00033C182F40401300E8227FBEC0AF01200A0
:1027F00084C3E8FF0F0BE83AE8CFB1F585C3E8FFE3
:102800000F0B0501B11387C3E8FF0F0BE83AE8CFC0
:10281000B0F588C3E8FF0F0B0501B0138AC3E8FFCA
:102820000F0BE83AE8CFAFF58BC3E8FF0F0B0501BC
:10283000AF138DC3E8FF0F0BE8CFAEF58FC3E8FFF2
:102840000F0BE83AE8CFADF590C3E8FF0F0B050199
:10285000AD1392C3E8FF0F0BE83AE8CFACF593C392
:10286000E8FF0F0B0501AC1395C3E8FF0F0BE83A27
:10287000E8CFABF596C3E8FF0F0B0501AB133CECBB
:102880002BF004014C0E826FFBEC0AF00401430EA6
:10289000826FFBEC0AF00AEF13F00784E9EC32F0E8
:1028A00024EC29F02DC500F1C7EC28F004014C0EF2
:1028B000826FFBEC0AF00401300E826FFBEC0AF031
:1028C00004012C0E826FFBEC0AF031C182F404018A
:1028D000300E8227FBEC0AF032C182F40401300E84
:1028E0008227FBEC0AF033C182F40401300E822708
:1028F000FBEC0AF004012C0E826FFBEC0AF024ECD6
:1029000029F02EC500F1C7EC28F031C182F4040192
:10291000300E8227FBEC0AF032C182F40401300E43
:102920008227FBEC0AF033C182F40401300E8227C7
:10293000FBEC0AF007948BEF19F004014C0E826F48
:10294000FBEC0AF00401650E826FFBEC0AF01CEC54
:102950002DF08BEF19F004014C0E826FFBEC0AF0A6
:102960000401450E826FFBEC0AF039EC2DF08BEF81
:1029700019F004014C0E826FFBEC0AF00401620EA8
:10298000826FFBEC0AF073EC2DF08BEF19F0040171
:102990004C0E826FFBEC0AF00401420E826FFBECDE
:1029A0000AF056EC2DF08BEF19F004014C0E826FFB
:1029B000FBEC0AF004015A0E826FFBEC0AF00401F2
:1029C0002C0E826FFBEC0AF0E9EC32F024EC29F0DB
:1029D00005012E51130A06E005012E51170A0DE0DC
:1029E00006EF15F00101000E006F000E016F100ED2
:1029F000026F000E036F06EF15F00101000E006F6D
:102A0000000E016F000E026F010E036F0101200E18
:102A1000046F000E056F000E066F000E076F5AEC74
:102A200028F0C7EC28F02AC182F40401300E822776
:102A3000FBEC0AF02BC182F40401300E8227FBEC80
:102A40000AF02CC182F40401300E8227FBEC0AF05C
:102A50002DC182F40401300E8227FBEC0AF02EC156
:102A600082F40401300E8227FBEC0AF02FC182F4BD
:102A70000401300E8227FBEC0AF030C182F404011D
:102A8000300E8227FBEC0AF031C182F40401300ED3
:102A90008227FBEC0AF032C182F40401300E822757
:102AA000FBEC0AF033C182F40401300E8227FBEC08
:102AB0000AF08BEF19F0078404014C0E826FFBECD7
:102AC0000AF00401310E826FFBEC0AF004012C0EB7
:102AD000826FFBEC0AF025C500F126C501F127C580
:102AE00002F128C503F10101200E046F000E056FED
:102AF000000E066F000E076F5AEC28F0C7EC28F0A6
:102B00002AC182F40401300E8227FBEC0AF02BC1AB
:102B100082F40401300E8227FBEC0AF02CC182F40F
:102B20000401300E8227FBEC0AF02DC182F404016F
:102B3000300E8227FBEC0AF02EC182F40401300E25
:102B40008227FBEC0AF02FC182F40401300E8227A9
:102B5000FBEC0AF030C182F40401300E8227FBEC5A
:102B60000AF031C182F40401300E8227FBEC0AF036
:102B700032C182F40401300E8227FBEC0AF033C12B
:102B800082F40401300E8227FBEC0AF007948BEFED
:102B900019F0078404014C0E826FFBEC0AF004016B
:102BA000320E826FFBEC0AF069EC2FF007948BEF8A
:102BB00019F0078404014C0E826FFBEC0AF004014B
:102BC000330E826FFBEC0AF0C6EC2FF0079466EF31
:102BD00015F0078404014C0E826FFBEC0AF004012F
:102BE000340E826FFBEC0AF004012C0E826FFBECBA
:102BF0000AF065EC29F084C32AF185C32BF186C362
:102C00002CF187C32DF188C32EF189C32FF18AC31C
:102C100030F18BC331F18CC332F18DC333F101013B
:102C2000296B72EC29F0E9EC28F0200E046F000EFD
:102C3000056F000E066F000E076F3AEC28F000C11A
:102C400021F501C122F502C123F503C124F59CEC55
:102C500032F034C5ABF535C5ACF536C5ADF537C585
:102C6000AEF538C5AFF539C5B0F53AC5B1F515ECD7
:102C700013F004012C0E826FFBEC0AF03BC500F14F
:102C80003CC501F13DC502F13EC503F10101000E55
:102C9000046F000E056F010E066F000E076F5AECF1
:102CA00028F0C7EC28F0296758EF16F05DEF16F012
:102CB00004012D0E826FFBEC0AF030C182F4040196
:102CC000300E8227FBEC0AF031C182F40401300E91
:102CD0008227FBEC0AF004012E0E826FFBEC0AF057
:102CE00032C182F40401300E8227FBEC0AF033C1BA
:102CF00082F40401300E8227FBEC0AF004012C0E52
:102D0000826FFBEC0AF024EC29F03FC500F140C5CE
:102D100001F1A0EC22F004012C0E826FFBEC0AF012
:102D200024EC29F041C500F1C7EC28F031C182F450
:102D30000401300E8227FBEC0AF032C182F4040158
:102D4000300E8227FBEC0AF033C182F40401300E0E
:102D50008227FBEC0AF004012C0E826FFBEC0AF0D8
:102D60000101036B026B48C501F147C500F101AFDA
:102D7000BFEF16F00101FF0E026FFF0E036FC7ECED
:102D800028F02967C6EF16F0CBEF16F004012D0EE0
:102D9000826FFBEC0AF02FC182F40401300E82270F
:102DA000FBEC0AF030C182F40401300E8227FBEC08
:102DB0000AF031C182F40401300E8227FBEC0AF0E4
:102DC00032C182F40401300E8227FBEC0AF033C1D9
:102DD00082F40401300E8227FBEC0AF004012C0E71
:102DE000826FFBEC0AF00101036B026B4AC501F133
:102DF00049C500F101AF02EF17F00101FF0E026FAC
:102E0000FF0E036FC7EC28F0296709EF17F00EEFEC
:102E100017F004012D0E826FFBEC0AF02FC182F433
:102E20000401300E8227FBEC0AF030C182F4040169
:102E3000300E8227FBEC0AF031C182F40401300E1F
:102E40008227FBEC0AF032C182F40401300E8227A3
:102E5000FBEC0AF033C182F40401300E8227FBEC54
:102E60000AF004012C0E826FFBEC0AF00101036BE7
:102E7000026B4CC501F14BC500F101AF45EF17F0F6
:102E80000101FF0E026FFF0E036FC7EC28F02967E8
:102E90004CEF17F051EF17F004012D0E826FFBEC91
:102EA0000AF02FC182F40401300E8227FBEC0AF0F5
:102EB00030C182F40401300E8227FBEC0AF031C1EC
:102EC00082F40401300E8227FBEC0AF032C182F456
:102ED0000401300E8227FBEC0AF033C182F40401B6
:102EE000300E8227FBEC0AF004012C0E826FFBEC03
:102EF0000AF00101036B026B4EC501F14DC500F1F3
:102F000001AF88EF17F00101FF0E026FFF0E036F94
:102F1000C7EC28F029678FEF17F094EF17F0040142
:102F20002D0E826FFBEC0AF02FC182F40401300EEB
:102F30008227FBEC0AF030C182F40401300E8227B4
:102F4000FBEC0AF031C182F40401300E8227FBEC65
:102F50000AF032C182F40401300E8227FBEC0AF041
:102F600033C182F40401300E8227FBEC0AF0040125
:102F70002C0E826FFBEC0AF00101036B026B50C553
:102F800001F14FC500F101AFCBEF17F00101FF0ECA
:102F9000026FFF0E036FC7EC28F02967D2EF17F01E
:102FA000D7EF17F004012D0E826FFBEC0AF02FC152
:102FB00082F40401300E8227FBEC0AF030C182F467
:102FC0000401300E8227FBEC0AF031C182F40401C7
:102FD000300E8227FBEC0AF032C182F40401300E7D
:102FE0008227FBEC0AF033C182F40401300E822701
:102FF000FBEC0AF004012C0E826FFBEC0AF00101DD
:10300000036B026B52C501F151C500F101AF0EEF28
:1030100018F00101FF0E026FFF0E036FC7EC28F0DE
:10302000296715EF18F01AEF18F004012D0E826FC2
:10303000FBEC0AF02FC182F40401300E8227FBEC76
:103040000AF030C182F40401300E8227FBEC0AF052
:1030500031C182F40401300E8227FBEC0AF032C148
:1030600082F40401300E8227FBEC0AF033C182F4B3
:103070000401300E8227FBEC0AF004012C0E826F53
:10308000FBEC0AF00101036B026B46C501F145C57B
:1030900000F101AF51EF18F00101FF0E026FFF0EBA
:1030A000036FC7EC28F0296758EF18F05DEF18F0B0
:1030B00004012D0E826FFBEC0AF02FC182F4040193
:1030C000300E8227FBEC0AF030C182F40401300E8E
:1030D0008227FBEC0AF031C182F40401300E822712
:1030E000FBEC0AF032C182F40401300E8227FBECC3
:1030F0000AF033C182F40401300E8227FBEC0AF09F
:1031000007948BEF19F065EC29F085C32AF186C38B
:103110002BF187C32CF188C32DF189C32EF18AC30B
:103120002FF18BC330F18CC331F18DC332F18EC3DB
:1031300033F10101296B72EC29F0E9EC28F001016F
:10314000010E046F000E056F000E066F000E076F74
:1031500029EC28F0100E046F000E056F000E066FAC
:10316000000E076F3AEC28F000C129F501C12AF5DD
:1031700002C12BF503C12CF5F2EC2EF004014C0E2C
:10318000826FFBEC0AF00401460E826FFBEC0AF042
:1031900004012C0E826FFBEC0AF025C500F126C558
:1031A00001F127C502F128C503F10101100E046FDA
:1031B000000E056F000E066F000E076F5AEC28F028
:1031C000C7EC28F02AC182F40401300E8227FBEC00
:1031D0000AF02BC182F40401300E8227FBEC0AF0C6
:1031E0002CC182F40401300E8227FBEC0AF02DC1C1
:1031F00082F40401300E8227FBEC0AF02EC182F427
:103200000401300E8227FBEC0AF02FC182F4040186
:10321000300E8227FBEC0AF030C182F40401300E3C
:103220008227FBEC0AF031C182F40401300E8227C0
:10323000FBEC0AF032C182F40401300E8227FBEC71
:103240000AF033C182F40401300E8227FBEC0AF04D
:103250008BEF19F00F98C6EC2FF076EF21F00401F8
:103260004C0E826FFBEC0AF00401350E826FFBEC12
:103270000AF004012C0E826FFBEC0AF024EC29F01A
:103280000784B5C500F10794C7EC28F031C182F47A
:103290000401300E8227FBEC0AF032C182F40401F3
:1032A000300E8227FBEC0AF033C182F40401300EA9
:1032B0008227FBEC0AF08BEF19F089EC2FF024EC5D
:1032C00029F033C500F1C7EC28F004014C0E826FE1
:1032D000FBEC0AF00401360E826FFBEC0AF00401ED
:1032E0002C0E826FFBEC0AF031C182F40401300E27
:1032F0008227FBEC0AF032C182F40401300E8227EF
:10330000FBEC0AF033C182F40401300E8227FBEC9F
:103310000AF08BEF19F005EC0BF076EF21F00401C9
:103320004C0E826FFBEC0AF00401500E826FFBEC36
:103330000AF004012C0E826FFBEC0AF085C32AF11F
:1033400086C32BF187C32CF188C32DF189C32EF1DD
:103350008AC32FF18BC330F18CC331F18DC332F1AD
:103360008EC333F1010172EC29F0E9EC28F003017E
:103370008451530A0DE0030184514D0A38E00401E1
:10338000780E826FFBEC0AF005EC0BF076EF21F083
:103390000401530E826FFBEC0AF0250E0C6E00C187
:1033A0000BF0EEEC07F0260E0C6E01C10BF0EEEC0C
:1033B00007F0270E0C6E02C10BF0EEEC07F0280EA2
:1033C0000C6E03C10BF0EEEC07F000C153F501C128
:1033D00054F502C155F503C156F500C157F501C1B9
:1033E00058F502C159F503C15AF56CEF1AF0040102
:1033F0004D0E826FFBEC0AF0290E0C6E00C10BF033
:10340000EEEC07F000C15BF500C15CF56CEF1AF063
:1034100004014C0E826FFBEC0AF00401540E826F23
:10342000FBEC0AF004012C0E826FFBEC0AF084C363
:103430002AF185C32BF186C32CF187C32DF188C3F4
:103440002EF189C32FF18AC330F18BC331F18DC3C3
:1034500032F18EC333F1010172EC29F0E9EC28F06E
:103460000101000E046F000E056F010E066F000EC5
:10347000076F3AEC28F0210E0C6E00C10BF0EEEC59
:1034800007F0220E0C6E01C10BF0EEEC07F0230EDC
:103490000C6E02C10BF0EEEC07F0240E0C6E03C1B3
:1034A0000BF0EEEC07F000C15DF501C15EF502C165
:1034B0005FF503C160F56CEF1AF004014C0E826FEA
:1034C000FBEC0AF00401490E826FFBEC0AF00401E8
:1034D0002C0E826FFBEC0AF0250E05EC08F0E8CF0D
:1034E00000F1260E05EC08F0E8CF01F1270E05ECFF
:1034F00008F0E8CF02F1280E05EC08F0E8CF03F160
:10350000C7EC28F0AAEC26F00401730E826FFBECE6
:103510000AF004012C0E826FFBEC0AF024EC29F077
:10352000290E05EC08F0E8CF00F1C7EC28F0AAEC72
:1035300026F00401730E826FFBEC0AF004012C0EDE
:10354000826FFBEC0AF057C500F158C501F159C56F
:1035500002F15AC503F1C7EC28F0AAEC26F00401E9
:10356000730E826FFBEC0AF004012C0E826FFBECF1
:103570000AF024EC29F05CC500F1C7EC28F0AAECB5
:1035800026F004016D0E826FFBEC0AF004012C0E94
:10359000826FFBEC0AF05DC500F15EC501F15FC50D
:1035A00002F160C503F191EC21F004012C0E826F51
:1035B000FBEC0AF005EC0BF076EF21F083C32AF167
:1035C00084C32BF185C32CF186C32DF187C32EF163
:1035D00088C32FF189C330F18AC331F18BC332F133
:1035E0008CC333F1010172EC29F0E9EC28F0160EDE
:1035F0000C6E00C10BF0EEEC07F0170E0C6E01C163
:103600000BF0EEEC07F0180E0C6E02C10BF0EEECB6
:1036100007F0190E0C6E03C10BF0EEEC07F000C1C1
:103620008AF101C18BF102C18CF103C18DF100C19E
:103630008EF101C18FF102C190F103C191F1C0EF90
:103640001BF083C32AF184C32BF185C32CF186C3FD
:103650002DF187C32EF188C32FF189C330F18AC3BE
:1036600031F18BC332F18CC333F1010172EC29F0DB
:10367000E9EC28F000C18AF101C18BF102C18CF1A3
:1036800003C18DF100C18EF101C18FF102C190F132
:1036900003C191F1C0EF1BF083C32AF184C32BF166
:1036A00085C32CF186C32DF187C32EF188C32FF17A
:1036B00089C330F18AC331F18CC332F18DC333F148
:1036C000010172EC29F0E9EC28F00101000E046F11
:1036D000000E056F010E066F000E076F3AEC28F022
:1036E0001A0E0C6E00C10BF0EEEC07F01B0E0C6E08
:1036F00001C10BF0EEEC07F01C0E0C6E02C10BF0DA
:10370000EEEC07F01D0E0C6E03C10BF0EEEC07F0B3
:1037100000C192F101C193F102C194F103C195F18D
:10372000C0EF1BF083C32AF184C32BF185C32CF1B6
:1037300086C32DF187C32EF188C32FF189C330F1E1
:103740008AC331F18CC332F18DC333F1010172ECC4
:1037500029F0E9EC28F00101000E046F000E056F5E
:10376000010E066F000E076F3AEC28F000C192F1CF
:1037700001C193F102C194F103C195F1C0EF1BF0B7
:10378000160E05EC08F0E8CF00F1170E05EC08F076
:10379000E8CF01F1180E05EC08F0E8CF02F1190EA0
:1037A00005EC08F0E8CF03F1C7EC28F0AAEC26F00E
:1037B0000401730E826FFBEC0AF004012C0E826F81
:1037C000FBEC0AF08AC100F18BC101F18CC102F15E
:1037D0008DC103F1C7EC28F0AAEC26F00401730EAA
:1037E000826FFBEC0AF004012C0E826FFBEC0AF0F6
:1037F0001A0E05EC08F0E8CF00F11B0E05EC08F0FE
:10380000E8CF01F11C0E05EC08F0E8CF02F11D0E27
:1038100005EC08F0E8CF03F191EC21F004012C0E47
:10382000826FFBEC0AF092C100F193C101F194C1E7
:1038300002F195C103F191EC21F005EC0BF076EF6C
:1038400021F00401690E826FFBEC0AF004012C0EDA
:10385000826FFBEC0AF00101040E006F000E016F95
:10386000000E026F000E036FC7EC28F02CC182F42B
:103870000401300E8227FBEC0AF02DC182F4040112
:10388000300E8227FBEC0AF02EC182F40401300EC8
:103890008227FBEC0AF02FC182F40401300E82274C
:1038A000FBEC0AF030C182F40401300E8227FBECFD
:1038B0000AF031C182F40401300E8227FBEC0AF0D9
:1038C00032C182F40401300E8227FBEC0AF033C1CE
:1038D00082F40401300E8227FBEC0AF004012C0E66
:1038E000826FFBEC0AF001010B0E006F000E016FFE
:1038F000000E026F000E036FC7EC28F02CC182F49B
:103900000401300E8227FBEC0AF02DC182F4040181
:10391000300E8227FBEC0AF02EC182F40401300E37
:103920008227FBEC0AF02FC182F40401300E8227BB
:10393000FBEC0AF030C182F40401300E8227FBEC6C
:103940000AF031C182F40401300E8227FBEC0AF048
:1039500032C182F40401300E8227FBEC0AF033C13D
:1039600082F40401300E8227FBEC0AF004012C0ED5
:10397000826FFBEC0AF001011E0E006F000E016F5A
:10398000000E026F000E036FC7EC28F02CC182F40A
:103990000401300E8227FBEC0AF02DC182F40401F1
:1039A000300E8227FBEC0AF02EC182F40401300EA7
:1039B0008227FBEC0AF02FC182F40401300E82272B
:1039C000FBEC0AF030C182F40401300E8227FBECDC
:1039D0000AF031C182F40401300E8227FBEC0AF0B8
:1039E00032C182F40401300E8227FBEC0AF033C1AD
:1039F00082F40401300E8227FBEC0AF004012C0E45
:103A0000826FFBEC0AF0200EF86EF76AF66A04018A
:103A10000900F5CF82F4FBEC0AF00900F5CF82F43F
:103A2000FBEC0AF00900F5CF82F4FBEC0AF0090088
:103A3000F5CF82F4FBEC0AF00900F5CF82F4FBEC41
:103A40000AF00900F5CF82F4FBEC0AF00900F5CF8B
:103A500082F4FBEC0AF00900F5CF82F4FBEC0AF0EB
:103A600005EC0BF076EF21F08351630AD8A476EFD2
:103A700021F08451610AD8A476EF21F085516C0AB7
:103A8000D8A476EF21F08651410A42E08651440ADB
:103A90001BE08651420AD8B49BEF1DF08651350ACF
:103AA000D8B400EF23F08651360AD8B455EF23F08E
:103AB0008651370AD8B4BEEF23F08651380AD8B4FD
:103AC0001CEF24F076EF21F00798079A04017A0E94
:103AD000826FFBEC0AF00401780E826FFBEC0AF0B7
:103AE0000401640E826FFBEC0AF081A87FEF1DF0E9
:103AF0000401550E826FFBEC0AF084EF1DF0040107
:103B00004C0E826FFBEC0AF005EC0BF076EF21F027
:103B10000788079A04017A0E826FFBEC0AF0040111
:103B2000410E826FFBEC0AF00401610E826FFBEC28
:103B30000AF075EF1DF00798078A04017A0E826F6C
:103B4000FBEC0AF00401420E826FFBEC0AF0040168
:103B5000610E826FFBEC0AF075EF1DF001016667E4
:103B6000B9EF1DF06767B9EF1DF06867B9EF1DF099
:103B70006967D1EF1DF04F67C5EF1DF05067C5EFC6
:103B80001DF05167C5EF1DF05267D1EF1DF0010127
:103B9000000E006F000E016F000E026F000E036F2B
:103BA00012000101620E046F010E056F000E066F18
:103BB000000E076F66C100F167C101F168C102F133
:103BC00069C103F129EC28F003BF55EF1EF0010194
:103BD000000E046FA80E056F550E066F020E076FDC
:103BE00066C100F167C101F168C102F169C103F169
:103BF00066C186F167C187F168C188F169C189F141
:103C000029EC28F003BF0EEF1EF00101000E866FB5
:103C1000A80E876F550E886F020E896F0E0E05EC89
:103C200008F0E8CF18F10F0E05EC08F0E8CF19F115
:103C3000100E05EC08F0E8CF1AF1110E05EC08F0B3
:103C4000E8CF1BF172EC27F086C104F187C105F1C2
:103C500088C106F189C107F129EC28F0078236EC0A
:103C600027F072EC27F0079236EC27F086C100F1BE
:103C700087C101F188C102F189C103F1079236ECD5
:103C800027F0CC0E046FE00E056F870E066F050E51
:103C9000076F29EC28F000C118F101C119F102C128
:103CA0001AF103C11BF18DEF1EF00101800E006FB0
:103CB0001A0E016F060E026F000E036F4FC104F162
:103CC00050C105F151C106F152C107F129EC28F0AC
:103CD00003AF6EEF1EF024EC29F012000E0E05EC7F
:103CE00008F0E8CF18F10F0E05EC08F0E8CF19F155
:103CF000100E05EC08F0E8CF1AF1110E05EC08F0F3
:103D0000E8CF1BF14FC100F150C101F151C102F1E7
:103D100052C103F1078236EC27F018C100F119C136
:103D200001F11AC102F11BC103F112000401730E6B
:103D3000826FFBEC0AF004012C0E826FFBEC0AF0A0
:103D4000078462C166F163C167F164C168F165C14E
:103D500069F14BC14FF14CC150F14DC151F14EC110
:103D600052F157C159F158C15AF10794BCEC1EF0F9
:103D700005EC0BF076EF21F066C100F167C101F1AF
:103D800068C102F169C103F10101C7EC28F0AAEC96
:103D900026F00401630E826FFBEC0AF004012C0E86
:103DA000826FFBEC0AF04FC100F150C101F151C12B
:103DB00002F152C103F10101C7EC28F0AAEC26F090
:103DC0000401660E826FFBEC0AF004012C0E826F78
:103DD000FBEC0AF024EC29F059C100F15AC101F1C1
:103DE0000101C7EC28F0AAEC26F00401740E826FE2
:103DF000FBEC0AF0120010820401530E826FFBEC00
:103E00000AF004012C0E826FFBEC0AF083C32AF146
:103E100084C32BF185C32CF186C32DF187C32EF10A
:103E200088C32FF189C330F18AC331F18BC332F1DA
:103E30008CC333F1010172EC29F0E9EC28F000C1E8
:103E400066F101C167F102C168F103C169F18EC376
:103E50002AF18FC32BF190C32CF191C32DF192C3A2
:103E60002EF193C32FF194C330F195C331F196C372
:103E700032F197C333F1010172EC29F0E9EC28F03B
:103E800000C14FF101C150F102C151F103C152F122
:103E900065EC29F099C32FF19AC330F19BC331F13E
:103EA0009CC332F19DC333F1010172EC29F0E9ECBE
:103EB00028F000C159F101C15AF1BCEC1EF0040117
:103EC0002C0E826FFBEC0AF06DEF1FF08251520A4C
:103ED00003E10F826DEF1FF00F928251750A03E12B
:103EE000108474EF1FF010948251550A03E110867C
:103EF0007BEF1FF01096078410B2D8EF1FF010A4CC
:103F0000C4EF1FF0B6C166F1B7C167F1B8C168F17F
:103F1000B9C169F1BAC16AF1BBC16BF1BCC16CF145
:103F2000BDC16DF1BEC16EF1BFC16FF1C0C170F115
:103F3000C1C171F1C2C172F1C3C173F1C4C174F1E5
:103F4000C5C175F1C6C176F1C7C177F1C8C178F1B5
:103F5000C9C179F1CAC17AF1CBC17BF1CCC17CF185
:103F6000CDC17DF1CEC17EF1CFC17FF1D0C180F155
:103F7000D1C181F1D2C182F1D3C183F1D4C184F125
:103F8000D5C185F1CCEF1FF062C166F163C167F165
:103F900064C168F165C169F14BC14FF14CC150F189
:103FA0004DC151F14EC152F157C159F158C15AF1A9
:103FB00007940FA0FAEF1FF001019267E7EF1FF0DF
:103FC0009367E7EF1FF09467E7EF1FF09567EBEF5C
:103FD0001FF0FAEF1FF0AEEC1DF092C104F193C197
:103FE00005F194C106F195C107F129EC28F003BF52
:103FF0003EEF21F0AEEC1DF00101000E046F000E4B
:10400000056F010E066F000E076F5AEC28F010A422
:1040100011EF20F00401750E826FFBEC0AF016EF31
:1040200020F00401720E826FFBEC0AF004012C0EEA
:10403000826FFBEC0AF0C7EC28F0296725EF20F02F
:104040000401200E826F28EF20F004012D0E826FF4
:10405000FBEC0AF030C182F40401300E8227FBEC45
:104060000AF031C182F40401300E8227FBEC0AF021
:1040700004012E0E826FFBEC0AF032C182F40401BF
:10408000300E8227FBEC0AF033C182F40401300EBB
:104090008227FBEC0AF004016D0E826FFBEC0AF044
:1040A00004012C0E826FFBEC0AF04FC100F150C1ED
:1040B00001F151C102F152C103F10101C7EC28F035
:1040C000AAEC26F00401480E826FFBEC0AF0040112
:1040D0007A0E826FFBEC0AF004012C0E826FFBEC6F
:1040E0000AF066C100F167C101F168C102F169C15E
:1040F00003F10101C7EC28F0AAEC26F00401630EDD
:10410000826FFBEC0AF004012C0E826FFBEC0AF0CC
:1041100066C100F167C101F168C102F169C103F133
:1041200001010A0E046F000E056F000E066F000EEF
:10413000076F3AEC28F0000E046F120E056F000EA8
:10414000066F000E076F5AEC28F0C7EC28F02AC162
:1041500082F40401300E8227FBEC0AF02BC182F4BA
:104160000401300E8227FBEC0AF02CC182F404011A
:10417000300E8227FBEC0AF02DC182F40401300ED0
:104180008227FBEC0AF02EC182F40401300E822754
:10419000FBEC0AF02FC182F40401300E8227FBEC05
:1041A0000AF030C182F40401300E8227FBEC0AF0E1
:1041B00004012E0E826FFBEC0AF031C182F404017F
:1041C000300E8227FBEC0AF032C182F40401300E7B
:1041D0008227FBEC0AF033C182F40401300E8227FF
:1041E000FBEC0AF00401730E826FFBEC0AF0040191
:1041F0002C0E826FFBEC0AF024EC29F059C100F17F
:104200005AC101F1A0EC22F00FB20AEF21F00FA089
:104210003CEF21F004012C0E826FFBEC0AF0200E23
:10422000F86EF76AF66A04010900F5CF82F4FBEC38
:104230000AF00900F5CF82F4FBEC0AF00900F5CF93
:1042400082F4FBEC0AF00900F5CF82F4FBEC0AF0F3
:104250000900F5CF82F4FBEC0AF00900F5CF82F4F7
:10426000FBEC0AF00900F5CF82F4FBEC0AF0090040
:10427000F5CF82F4FBEC0AF005EC0BF00F9076EF33
:1042800021F00401630E826FFBEC0AF004012C0E96
:10429000826FFBEC0AF07CEC21F004012C0E826FA3
:1042A000FBEC0AF0EFEC21F004012C0E826FFBEC2A
:1042B0000AF06BEC22F004012C0E826FFBEC0AF08A
:1042C0000101F80E006FCD0E016F660E026F030E36
:1042D000036F91EC21F004012C0E826FFBEC0AF0CD
:1042E00081EC22F005EC0BF076EF21F00301C26BBC
:1042F0000790109285EF24F0D8900E0E05EC08F090
:10430000E8CF00F10F0E05EC08F0E8CF01F1100E38
:1043100005EC08F0E8CF02F1110E05EC08F0E8CF4B
:1043200003F10101000E046F000E056F010E066F10
:10433000000E076F5AEC28F0C7EC28F02AC182F46F
:104340000401300E8227FBEC0AF02BC182F4040139
:10435000300E8227FBEC0AF02CC182F40401300EEF
:104360008227FBEC0AF02DC182F40401300E822773
:10437000FBEC0AF02EC182F40401300E8227FBEC24
:104380000AF02FC182F40401300E8227FBEC0AF000
:1043900030C182F40401300E8227FBEC0AF031C1F7
:1043A00082F40401300E8227FBEC0AF004012E0E89
:1043B000826FFBEC0AF032C182F40401300E8227D6
:1043C000FBEC0AF033C182F40401300E8227FBECCF
:1043D0000AF004016D0E826FFBEC0AF01200120E5F
:1043E00005EC08F0E8CF00F1130E05EC08F0E8CF7B
:1043F00001F1140E05EC08F0E8CF02F1150E05EC02
:1044000008F0E8CF03F101010A0E046F000E056FFA
:10441000000E066F000E076F3AEC28F0000E046FD6
:10442000120E056F000E066F000E076F5AEC28F093
:10443000C7EC28F02AC182F40401300E8227FBEC7D
:104440000AF02BC182F40401300E8227FBEC0AF043
:104450002CC182F40401300E8227FBEC0AF02DC13E
:1044600082F40401300E8227FBEC0AF02EC182F4A4
:104470000401300E8227FBEC0AF02FC182F4040104
:10448000300E8227FBEC0AF030C182F40401300EBA
:104490008227FBEC0AF004012E0E826FFBEC0AF07F
:1044A00031C182F40401300E8227FBEC0AF032C1E4
:1044B00082F40401300E8227FBEC0AF033C182F44F
:1044C0000401300E8227FBEC0AF00401730E826FA8
:1044D000FBEC0AF012000A0E05EC08F0E8CF00F140
:1044E0000B0E05EC08F0E8CF01F10C0E05EC08F01E
:1044F000E8CF02F10D0E05EC08F0E8CF03F1A0EFD4
:1045000022F0060E05EC08F0E8CF00F1070E05ECEE
:1045100008F0E8CF01F1080E05EC08F0E8CF02F151
:10452000090E05EC08F0E8CF03F1A0EF22F001013D
:1045300024EC29F0078457C100F158C101F1079418
:104540000101E80E046F800E056F000E066F000E6D
:10455000076F3AEC28F0000E046F040E056F000E92
:10456000066F000E076F5AEC28F0880E046F130ECA
:10457000056F000E066F000E076F29EC28F00A0E7B
:10458000046F000E056F000E066F000E076F5AECE9
:1045900028F0C7EC28F001012967D4EF22F00401CC
:1045A000200E826FD7EF22F004012D0E826FFBECFC
:1045B0000AF030C182F40401300E8227FBEC0AF0CD
:1045C00031C182F40401300E8227FBEC0AF032C1C3
:1045D00082F40401300E8227FBEC0AF004012E0E57
:1045E000826FFBEC0AF033C182F40401300E8227A3
:1045F000FBEC0AF00401430E826FFBEC0AF01200A0
:1046000087C32AF188C32BF189C32CF18AC32DF10A
:104610008BC32EF18CC32FF18DC330F18EC331F1DA
:1046200090C332F191C333F10101296B72EC29F08F
:10463000E9EC28F00101000E046F000E056F010E79
:10464000066F000E076F3AEC28F00E0E0C6E00C1DC
:104650000BF0EEEC07F00F0E0C6E01C10BF0EEEC60
:1046600007F0100E0C6E02C10BF0EEEC07F0110E0D
:104670000C6E03C10BF0EEEC07F004017A0E826FB2
:10468000FBEC0AF004012C0E826FFBEC0AF0040133
:10469000350E826FFBEC0AF004012C0E826FFBECEE
:1046A0000AF07CEC21F084EF1DF087C32AF188C367
:1046B0002BF189C32CF18AC32DF18BC32EF18CC34E
:1046C0002FF18DC330F18EC331F190C332F191C31C
:1046D00033F10101296B72EC29F0E9EC28F0880E26
:1046E000046F130E056F000E066F000E076F2EECA1
:1046F00028F0000E046F040E056F000E066F000E0A
:10470000076F3AEC28F00101E80E046F800E056F88
:10471000000E066F000E076F5AEC28F00A0E0C6EA2
:1047200000C10BF0EEEC07F00B0E0C6E01C10BF0AC
:10473000EEEC07F00C0E0C6E02C10BF0EEEC07F085
:104740000D0E0C6E03C10BF0EEEC07F004017A0EB7
:10475000826FFBEC0AF004012C0E826FFBEC0AF076
:104760000401360E826FFBEC0AF004012C0E826FFE
:10477000FBEC0AF06BEC22F084EF1DF087C32AF10A
:1047800088C32BF189C32CF18AC32DF18BC32EF181
:104790008CC32FF18DC330F18FC331F190C332F14F
:1047A00091C333F1010172EC29F0E9EC28F0000E1D
:1047B000046F120E056F000E066F000E076F3AECC5
:1047C00028F001010A0E046F000E056F000E066F3F
:1047D000000E076F5AEC28F0120E0C6E00C10BF0A1
:1047E000EEEC07F0130E0C6E01C10BF0EEEC07F0CF
:1047F000140E0C6E02C10BF0EEEC07F0150E0C6EF1
:1048000003C10BF0EEEC07F004017A0E826FFBECB3
:104810000AF004012C0E826FFBEC0AF00401370E43
:10482000826FFBEC0AF004012C0E826FFBEC0AF0A5
:10483000EFEC21F084EF1DF087C32AF188C32BF140
:1048400089C32CF18AC32DF18BC32EF18CC32FF1B8
:104850008DC330F18EC331F190C332F191C333F186
:104860000101296B72EC29F0E9EC28F0880E046F45
:10487000130E056F000E066F000E076F2EEC28F06A
:10488000000E046F040E056F000E066F000E076F1A
:104890003AEC28F00101E80E046F800E056F000E5F
:1048A000066F000E076F5AEC28F0060E0C6E00C162
:1048B0000BF0EEEC07F0070E0C6E01C10BF0EEEC06
:1048C00007F0080E0C6E02C10BF0EEEC07F0090EBB
:1048D0000C6E03C10BF0EEEC07F004017A0E826F50
:1048E000FBEC0AF004012C0E826FFBEC0AF00401D1
:1048F000380E826FFBEC0AF004012C0E826FFBEC89
:104900000AF081EC22F084EF1DF081A843EF25F03E
:1049100007A8FCEF24F00101800E006F1A0E016F52
:10492000060E026F000E036F4BC104F14CC105F17E
:104930004DC106F14EC107F129EC28F003BF43EF4A
:1049400025F0A4EC26F04BC100F14CC101F14DC1A2
:1049500002F14EC103F1078236EC27F018C104F1D1
:1049600019C105F11AC106F11BC107F1F80E006F5C
:10497000CD0E016F660E026F030E036F29EC28F057
:104980000E0E0C6E00C10BF0EEEC07F00F0E0C6E6D
:1049900001C10BF0EEEC07F0100E0C6E02C10BF033
:1049A000EEEC07F0110E0C6E03C10BF0EEEC07F00D
:1049B0000784010124EC29F057C100F158C101F12D
:1049C00007940A0E0C6E00C10BF0EEEC07F00B0E14
:1049D0000C6E01C10BF0EEEC07F00C0E0C6E02C178
:1049E0000BF0EEEC07F00D0E0C6E03C10BF0EEECCD
:1049F00007F0079843EF25F007AA43EF25F0078457
:104A0000010124EC29F057C100F158C101F10794CC
:104A1000060E0C6E00C10BF0EEEC07F0070E0C6EEC
:104A200001C10BF0EEEC07F0080E0C6E02C10BF0AA
:104A3000EEEC07F0090E0C6E03C10BF0EEEC07F084
:104A4000078462C100F163C101F164C102F165C173
:104A500003F10794120E0C6E00C10BF0EEEC07F0A0
:104A6000130E0C6E01C10BF0EEEC07F0140E0C6E81
:104A700002C10BF0EEEC07F0150E0C6E03C10BF04B
:104A8000EEEC07F0079A0401805181197F0B0BE0CF
:104A90009EA809D014EE00F081517F0BE126E7506B
:104AA000812B0F01AD6E05012F51010A13E081AA80
:104AB0006AEF25F005012F51000A0AE00FB86AEFEE
:104AC00025F0050130676AEF25F00FB86AEF25F091
:104AD00028EF33F081B87FEF25F08DEC2BF0050146
:104AE0002F51020A02E07FEF25F05C2F7FEF25F0C7
:104AF0005BC55CF50501010E306F3C0E316F64EF54
:104B00000AF006013251385D3351D8A0010F395DEA
:104B1000800BD8A490EF25F032C638F633C639F6AC
:104B2000120006013251365D3351D8A0010F375DB6
:104B3000800BD8B4A0EF25F032C636F633C637F670
:104B4000120007841AC632F61BC633F61CC638F6A6
:104B50001DC639F681EC25F01EC632F61FC633F6A7
:104B600081EC25F020C632F621C633F681EC25F023
:104B70001AC632F61BC633F61CC636F61DC637F605
:104B800091EC25F01EC632F61FC633F691EC25F0E7
:104B900020C632F621C633F691EC25F03851365F47
:104BA0003951D8A03929375F24EC29F036C600F1F5
:104BB00037C601F130EC29F000C13AF601C13BF6ED
:104BC00022C632F623C633F624C638F625C639F691
:104BD00081EC25F026C632F627C633F681EC25F0A7
:104BE00028C632F629C633F681EC25F022C632F605
:104BF00023C633F624C636F625C637F691EC25F0E3
:104C000026C632F627C633F691EC25F028C632F6D2
:104C100029C633F691EC25F03851365F3951D8A0CA
:104C20003929375F24EC29F036C600F137C601F187
:104C300030EC29F000C13CF601C13DF62AC632F63F
:104C40002BC633F62CC638F62DC639F681EC25F086
:104C50002EC632F62FC633F681EC25F030C632F67A
:104C600031C633F681EC25F02AC632F62BC633F670
:104C70002CC636F62DC637F691EC25F02EC632F648
:104C80002FC633F691EC25F030C632F631C633F636
:104C900091EC25F03851365F3951D8A03929375F6A
:104CA00024EC29F036C600F137C601F130EC29F0CA
:104CB00000C13EF601C13FF63AC632F63BC633F6B6
:104CC0003CC636F63DC637F691EC25F03EC632F6C8
:104CD0003FC633F691EC25F00794120018C100F19D
:104CE00019C101F11AC102F11BC103F1000E046FD9
:104CF000000E056F010E066F000E076F5AEC28F0CC
:104D000029A199EF26F02051D8B499EF26F018C1C7
:104D100000F119C101F11AC102F11BC103F1000E2A
:104D2000046F000E056F0A0E066F000E076F5AEC37
:104D300028F012000101045100130551011306511E
:104D400002130751031312000101186B196B1A6B40
:104D50001B6B12002AC182F40401300E8227FBEC87
:104D60000AF02BC182F40401300E8227FBEC0AF01A
:104D70002CC182F40401300E8227FBEC0AF02DC115
:104D800082F40401300E8227FBEC0AF02EC182F47B
:104D90000401300E8227FBEC0AF02FC182F40401DB
:104DA000300E8227FBEC0AF030C182F40401300E91
:104DB0008227FBEC0AF031C182F40401300E822715
:104DC000FBEC0AF032C182F40401300E8227FBECC6
:104DD0000AF033C182F40401300E8227FBEC0AF0A2
:104DE00012002FC182F40401300E8227FBEC0AF07E
:104DF00030C182F40401300E8227FBEC0AF031C18D
:104E000082F40401300E8227FBEC0AF032C182F4F6
:104E10000401300E8227FBEC0AF033C182F4040156
:104E2000300E8227FBEC0AF01200060E116E060E01
:104E3000126E060E136E112E1BEF27F0122E1BEFB3
:104E400027F0132E1BEF27F08B84020E116E020E3B
:104E5000126E020E136E112E2BEF27F0122E2BEF77
:104E600027F0132E2BEF27F08B9412000101005333
:104E700005E1015303E1025301E1002BF9EC27F0B6
:104E800024EC29F03951006F3A51016F420E046F42
:104E90004B0E056F000E066F000E076F3AEC28F000
:104EA00000C104F101C105F102C106F103C107F11E
:104EB00018C100F119C101F11AC102F11BC103F1BE
:104EC00007B267EF27F02EEC28F069EF27F029EC06
:104ED00028F000C118F101C119F102C11AF103C192
:104EE0001BF1120024EC29F059C100F15AC101F163
:104EF000060E05EC08F0E8CF04F1070E05EC08F00B
:104F0000E8CF05F1080E05EC08F0E8CF06F1090E30
:104F100005EC08F0E8CF07F129EC28F000C124F1F6
:104F200001C125F102C126F103C127F1290E046F49
:104F3000000E056F000E066F000E076F3AEC28F0AA
:104F4000EE0E046F430E056F000E066F000E076F26
:104F50002EEC28F024C104F125C105F126C106F18B
:104F600027C107F13AEC28F000C11CF101C11DF185
:104F700002C11EF103C11FF1120E05EC08F0E8CFCB
:104F800004F1130E05EC08F0E8CF05F1140E05EC62
:104F900008F0E8CF06F1150E05EC08F0E8CF07F1B0
:104FA0000D0E006F000E016F000E026F000E036FFA
:104FB0003AEC28F0180E046F000E056F000E066F15
:104FC000000E076F5AEC28F01CC104F11DC105F159
:104FD0001EC106F11FC107F12EEC28F06A0E046F06
:104FE0002A0E056F000E066F000E076F29EC28F0E1
:104FF0001200BF0EFA6E200E3A6F396BD890003750
:10500000013702370337D8B00AEF28F03A2FFFEF05
:1050100027F039073A070353D8B412000331070BBE
:1050200080093F6F03390F0B010F396F80EC5FF080
:10503000406F390580EC5FF0405D405F396B3F3376
:10504000D8B0392739333FA91FEF28F0405139270D
:105050001200010149EC29F0D8B0120001010351FE
:105060000719346F0CEC29F0D8900751031934AFAD
:10507000800F12000101346B30EC29F0D8A046EC0F
:1050800029F0D8B012001BEC29F024EC29F01F0EF7
:10509000366F5CEC29F00B35D8B00CEC29F0D8A0B9
:1050A0000335D8B01200362F49EF28F034B133EC75
:1050B00029F012000101346B04510511061107118A
:1050C0000008D8A030EC29F0D8A046EC29F0D8B0E0
:1050D0001200086B096B0A6B0B6B5CEC29F01F0E5E
:1050E000366F5CEC29F007510B5DD8A484EF28F0F3
:1050F00006510A5DD8A484EF28F00551095DD8A4B3
:1051000084EF28F00451085DD8A097EF28F00451EF
:10511000085F0551D8A0053D095F0651D8A0063D9E
:105120000A5F0751D8A0073D0B5FD8900081362F4A
:1051300071EF28F034B133EC29F0346B30EC29F006
:10514000D89060EC29F007510B5DD8A4B4EF28F09B
:1051500006510A5DD8A4B4EF28F00551095DD8A422
:10516000B4EF28F00451085DD8A0C3EF28F0003F49
:10517000C3EF28F0013FC3EF28F0023FC3EF28F050
:10518000032BD8B4120034B133EC29F01200010122
:10519000346B30EC29F0D8B0120065EC29F0200E09
:1051A000366F003701370237033711EE33F00A0E3E
:1051B000376FE7360A0EE75CD8B0E76EE552372F57
:1051C000D9EF28F0362FD1EF28F034B12981D890CB
:1051D000120001010A0E346F200E366F11EE29F015
:1051E0003451376F0A0ED890E652D8B0E726E7322E
:1051F000372FF4EF28F00333023301330033362F17
:10520000EEEF28F0E750FF0FD8A00335D8B012001A
:1052100029B133EC29F01200045100270551D8B010
:10522000053D01270651D8B0063D02270751D8B0E9
:10523000073D032712000051086F0151096F025109
:105240000A6F03510B6F12000101006B016B026BBF
:10525000036B12000101046B056B066B076B1200F8
:105260000335D8A012000351800B001F011F021F3D
:10527000031F003F43EF29F0013F43EF29F0023FB6
:1052800043EF29F0032B342B032512000735D8A058
:1052900012000751800B041F051F061F071F043F44
:1052A00059EF29F0053F59EF29F0063F59EF29F052
:1052B000072B342B0725120000370137023703373D
:1052C000083709370A370B3712000101296B2A6B9F
:1052D0002B6B2C6B2D6B2E6B2F6B306B316B326B02
:1052E000336B120001012A510F0B2A6F2B510F0B48
:1052F0002B6F2C510F0B2C6F2D510F0B2D6F2E512F
:105300000F0B2E6F2F510F0B2F6F30510F0B306F74
:1053100031510F0B316F32510F0B326F33510F0B75
:10532000336F1200899C000EC76E200EC66E9E96CB
:10533000C69EC50EC96EFF0E9EB602D0E82EFCD7E3
:105340009E96C69E000EC96EFF0E9EB602D0E82E37
:10535000FCD7C9CF00F69E96C69E000EC96EFF0E02
:105360009EB602D0E82EFCD7C9CF01F6898C120078
:10537000000EC76E200EC66E899C9E96C69EC80EF5
:10538000C96EFF0E9EB602D0E82EFCD79E96C69E32
:10539000000EC96EFF0E9EB602D0E82EFCD7C9CF14
:1053A00002F69E96C69E000EC96EFF0E9EB602D0F5
:1053B000E82EFCD7C9CF03F6898C899C9E96C69EA1
:1053C000CA0EC96EFF0E9EB602D0E82EFCD79E967E
:1053D000C69E000EC96EFF0E9EB602D0E82EFCD708
:1053E000C9CF0AF69E96C69E000EC96EFF0E9EB6E7
:1053F00002D0E82EFCD7C9CF0BF6898C899C9E96EB
:10540000C69ECC0EC96EFF0E9EB602D0E82EFCD70B
:105410009E96C69E000EC96EFF0E9EB602D0E82E66
:10542000FCD7C9CF12F69E96C69E000EC96EFF0E1F
:105430009EB602D0E82EFCD7C9CF13F6898C120095
:10544000000EC76E200EC66E899C9E96C69EE80E04
:10545000C96EFF0E9EB602D0E82EFCD79E96C69E61
:10546000000EC96EFF0E9EB602D0E82EFCD7C9CF43
:105470001AF69E96C69E000EC96EFF0E9EB602D00C
:10548000E82EFCD7C9CF1BF6898C899C9E96C69EB8
:10549000EA0EC96EFF0E9EB602D0E82EFCD79E968D
:1054A000C69E000EC96EFF0E9EB602D0E82EFCD737
:1054B000C9CF22F69E96C69E000EC96EFF0E9EB6FE
:1054C00002D0E82EFCD7C9CF23F6898C899C9E9602
:1054D000C69EEC0EC96EFF0E9EB602D0E82EFCD71B
:1054E0009E96C69E000EC96EFF0E9EB602D0E82E96
:1054F000FCD7C9CF2AF69E96C69E000EC96EFF0E37
:105500009EB602D0E82EFCD7C9CF2BF6898C1200AC
:10551000000EC76E200EC66E899C9E96C69E240EF7
:10552000C96EFF0E9EB602D0E82EFCD79E96C69E90
:10553000E40EC96EFF0E9EB602D0E82EFCD7898C11
:10554000899C9E96C69E200EC96EFF0E9EB602D006
:10555000E82EFCD79E96C69E5F0EC96EFF0E9EB6C5
:1055600002D0E82EFCD7898C899C9E96C69E210E7F
:10557000C96EFF0E9EB602D0E82EFCD79E96C69E40
:10558000C00EC96EFF0E9EB602D0E82EFCD7898CE5
:10559000899C9E96C69E260EC96EFF0E9EB602D0B0
:1055A000E82EFCD79E96C69E000EC96EFF0E9EB6D4
:1055B00002D0E82EFCD7898C12008984000EC76EB9
:1055C000220EC66E9E96C69E000EC96EFF0E9EB639
:1055D00002D0E82EFCD79E96C69E000EC96EFF0E26
:1055E0009EB602D0E82EFCD7C9CFABF59E96C69EDC
:1055F000000EC96EFF0E9EB602D0E82EFCD7C9CFB2
:10560000ACF59E96C69E000EC96EFF0E9EB602D0E9
:10561000E82EFCD7C9CFADF59E96C69E000EC96E8A
:10562000FF0E9EB602D0E82EFCD7C9CFAEF59E96EF
:10563000C69E000EC96EFF0E9EB602D0E82EFCD7A5
:10564000C9CFAFF59E96C69E000EC96EFF0E9EB6E0
:1056500002D0E82EFCD7C9CFB0F59E96C69E000EAC
:10566000C96EFF0E9EB602D0E82EFCD7C9CFB1F5A9
:10567000899490EC2DF012008984000EC76E220EE2
:10568000C66E9E96C69E800EC96EFF0E9EB602D056
:10569000E82EFCD79E96C69EABC5C9FFFF0E9EB6F0
:1056A00002D0E82EFCD79E96C69EACC5C9FFFF0E61
:1056B0009EB602D0E82EFCD79E96C69EADC5C9FF09
:1056C000FF0E9EB602D0E82EFCD79E96C69EAEC5B3
:1056D000C9FFFF0E9EB602D0E82EFCD79E96C69E4E
:1056E000AFC5C9FFFF0E9EB602D0E82EFCD79E962E
:1056F000C69EB0C5C9FFFF0E9EB602D0E82EFCD7ED
:105700009E96C69EB1C5C9FFFF0E9EB602D0E82E7A
:10571000FCD7899490EC2DF012008984000EC76E9E
:10572000220EC66E9E96C69E070EC96EFF0E9EB6D0
:1057300002D0E82EFCD79E96C69E000EC96EFF0EC4
:105740009EB602D0E82EFCD7C9CFABF59E96C69E7A
:10575000000EC96EFF0E9EB602D0E82EFCD7C9CF50
:10576000ACF59E96C69E000EC96EFF0E9EB602D088
:10577000E82EFCD7C9CFADF59E96C69E000EC96E29
:10578000FF0E9EB602D0E82EFCD7C9CFAEF58994A5
:1057900090EC2DF08984000EC76E220EC66E9E9688
:1057A000C69E0F0EC96EFF0E9EB602D0E82EFCD725
:1057B0009E96C69E000EC96EFF0E9EB602D0E82EC3
:1057C000FCD7C9CFB3F5899490EC2DF012008984F1
:1057D000000EC76E220EC66E9E96C69E870EC96EBE
:1057E000FF0E9EB602D0E82EFCD79E96C69EABC595
:1057F000C9FFFF0E9EB602D0E82EFCD79E96C69E2D
:10580000ACC5C9FFFF0E9EB602D0E82EFCD79E960F
:10581000C69EADC5C9FFFF0E9EB602D0E82EFCD7CE
:105820009E96C69EAEC5C9FFFF0E9EB602D0E82E5C
:10583000FCD7899490EC2DF089849E96C69E8F0E9D
:10584000C96EFF0E9EB602D0E82EFCD79E96C69E6D
:10585000B3C5C9FFFF0E9EB602D0E82EFCD78994CF
:1058600090EC2DF012008984000EC76E220EC66ED9
:105870009E96C69E870EC96EFF0E9EB602D0E82E7B
:10588000FCD79E96C69E000EC96EFF0E9EB602D035
:10589000E82EFCD79E96C69E800EC96EFF0E9EB661
:1058A00002D0E82EFCD79E96C69E800EC96EFF0ED3
:1058B0009EB602D0E82EFCD79E96C69E800EC96E7C
:1058C000FF0E9EB602D0E82EFCD7899490EC2DF006
:1058D00089849E96C69E8F0EC96EFF0E9EB602D01C
:1058E000E82EFCD79E96C69E010EC96EFF0E9EB690
:1058F00002D0E82EFCD7899490EC2DF01200898418
:10590000000EC76E220EC66E9E96C69E870EC96E8C
:10591000FF0E9EB602D0E82EFCD79E96C69E000EC5
:10592000C96EFF0E9EB602D0E82EFCD79E96C69E8C
:10593000000EC96EFF0E9EB602D0E82EFCD79E96D2
:10594000C69E800EC96EFF0E9EB602D0E82EFCD712
:105950009E96C69E800EC96EFF0E9EB602D0E82EA1
:10596000FCD7899490EC2DF089849E96C69E8F0E6C
:10597000C96EFF0E9EB602D0E82EFCD79E96C69E3C
:10598000010EC96EFF0E9EB602D0E82EFCD7899498
:1059900090EC2DF012008984000EC76E220EC66EA8
:1059A0009E96C69E8F0EC96EFF0E9EB602D0E82E42
:1059B000FCD790EC2DF09E96C69E810EC96EFF0E10
:1059C0009EB602D0E82EFCD7899490EC2DF0898405
:1059D000000EC76E220EC66E9E96C69E8F0EC96EB4
:1059E000FF0E9EB602D0E82EFCD790EC2DF09E96CE
:1059F000C69E010EC96EFF0E9EB602D0E82EFCD7E1
:105A0000899490EC2DF089849E96C69E910EC96E65
:105A1000FF0E9EB602D0E82EFCD790EC2DF09E969D
:105A2000C69EA50EC96EFF0E9EB602D0E82EFCD70C
:105A3000899490EC2DF012008984000EC76E220E1E
:105A4000C66E9E96C69E8F0EC96EFF0E9EB602D083
:105A5000E82EFCD790EC2DF09E96C69E810EC96E66
:105A6000FF0E9EB602D0E82EFCD7899490EC2DF064
:105A700012008984000EC76E220EC66E9E96C69EC8
:105A80008F0EC96EFF0E9EB602D0E82EFCD790ECAA
:105A90002DF09E96C69E010EC96EFF0E9EB602D0D8
:105AA000E82EFCD7899490EC2DF012008984000E2A
:105AB000C76E220EC66E9E96C69E910EC96EFF0ED2
:105AC0009EB602D0E82EFCD790EC2DF09E96C69E96
:105AD000A50EC96EFF0E9EB602D0E82EFCD78994A3
:105AE00090EC2DF012008984000EC76E220EC66E57
:105AF0009E96C69E910EC96EFF0E9EB602D0E82EEF
:105B0000FCD790EC2DF09E96C69E000EC96EFF0E3F
:105B10009EB602D0E82EFCD7899490EC2DF01200AE
:105B2000050EE82EFED712000501256B266B276BAC
:105B3000286B899A400EC76E200EC66E9E96C69E32
:105B4000030EC96EFF0E9EB602D0E82EFCD79E96BD
:105B5000C69E27C5C9FFFF0E9EB602D0E82EFCD711
:105B60009E96C69E26C5C9FFFF0E9EB602D0E82EA1
:105B7000FCD79E96C69E25C5C9FFFF0E9EB602D0D5
:105B8000E82EFCD79E96C69EC952FF0E9EB602D046
:105B9000E82EFCD7898A0F01C950FF0A01E11200E3
:105BA00005012E51130A05E005012E51170A0CE0DC
:105BB00012000501E00E256FFF0E266F0F0E276FF6
:105BC000000E286FEDEF2DF00501E00E256FFF0EA2
:105BD000266FFF0E276F000E286F899A400EC76E42
:105BE000200EC66E9E96C69E030EC96EFF0E9EB612
:105BF00002D0E82EFCD79E96C69E27C5C9FFFF0E91
:105C00009EB602D0E82EFCD79E96C69E26C5C9FF3A
:105C1000FF0E9EB602D0E82EFCD79E96C69E25C5E6
:105C2000C9FFFF0E9EB602D0E82EFCD79E96C69EF8
:105C3000C952FF0E9EB602D0E82EFCD7898A0F010A
:105C4000C950FF0A1DE005012E51130A05E00501A8
:105C50002E51170A0BE012000501000E256F000EF1
:105C6000266F100E276F000E286F12000501000E20
:105C7000256F000E266F000E276F010E286F120091
:105C80000501256B266B276B286B05012E51130A26
:105C900005E005012E51170A0CE012000501000E67
:105CA000216F000E226F040E236F000E246F62EF2F
:105CB0002EF00501000E216F000E226F800E236F63
:105CC000000E246F21C500F122C501F123C502F1A8
:105CD00024C503F125C504F126C505F127C506F144
:105CE00028C507F19AEC26F000C125F501C126F57B
:105CF00002C127F503C128F5899A400EC76E200E10
:105D0000C66E9E96C69E030EC96EFF0E9EB602D04C
:105D1000E82EFCD79E96C69E27C5C9FFFF0E9EB6ED
:105D200002D0E82EFCD79E96C69E26C5C9FFFF0E60
:105D30009EB602D0E82EFCD79E96C69E25C5C9FF0A
:105D4000FF0E9EB602D0E82EFCD79E96C69EC95284
:105D5000FF0E9EB602D0E82EFCD7898AC950FF0AF2
:105D600008E104C125F505C126F506C127F507C1DF
:105D700028F5D890050124332333223321332151D0
:105D8000E00B216F2167CCEF2EF02267CCEF2EF0D5
:105D90002367CCEF2EF0246762EF2EF00501200E72
:105DA0002527E86A2623E86A2723E86A28231200C1
:105DB000E86A05012E51130A06E005012E51170A63
:105DC0000BE0020E120005012851000A03E12751E1
:105DD000F00B07E0010E120005012851000A01E056
:105DE000010E120029C500F12AC501F12BC502F1EF
:105DF0002CC503F125C504F126C505F127C506F11B
:105E000028C507F129EC28F003BF1200D8EC2EF0CA
:105E10005FE1899A400EC76E200EC66E9E96C69EA2
:105E2000060EC96EFF0E9EB602D0E82EFCD7898AF8
:105E3000899A9E96C69E020EC96EFF0E9EB602D02D
:105E4000E82EFCD79E96C69E27C5C9FFFF0E9EB6BC
:105E500002D0E82EFCD79E96C69E26C5C9FFFF0E2F
:105E60009EB602D0E82EFCD79E96C69E25C5C9FFD9
:105E7000FF0E9EB602D0E82EFCD79E96C69E000E60
:105E8000C96EFF0E9EB602D0E82EFCD7898A899A89
:105E90009E96C69E050EC96EFF0E9EB602D0E82ED7
:105EA000FCD79E96C69EC952FF0E9EB602D0E82E23
:105EB000FCD7C9B051EF2FF0898A0501200E2527A4
:105EC000E86A2623E86A2723E86A2823F2EF2EF0FF
:105ED0001200899A400EC76E200EC66E9E96C69E10
:105EE000060EC96EFF0E9EB602D0E82EFCD7898A38
:105EF000899A9E96C69EC70EC96EFF0E9EB602D0A8
:105F0000E82EFCD7898A0501256B266B276B286B49
:105F10001200899A400EC76E200EC66E9E96C69ECF
:105F2000050EC96EFF0E9EB602D0E82EFCD79E96D7
:105F3000C69EC952FF0E9EB602D0E82EFCD7C9CF2E
:105F400033F5898A1200899A400EC76E200EC66EFC
:105F50009E96C69EB90EC96EFF0E9EB602D0E82E62
:105F6000FCD7898A1200899A400EC76E200EC66E31
:105F70009E96C69EAB0EC96EFF0E9EB602D0E82E50
:105F8000FCD7898AFF0EE82EFED71200D8EC2EF03F
:105F9000D8A41200899A400EC76E200EC66E9E9637
:105FA000C69E030EC96EFF0E9EB602D0E82EFCD729
:105FB0009E96C69E27C5C9FFFF0E9EB602D0E82E4C
:105FC000FCD79E96C69E26C5C9FFFF0E9EB602D080
:105FD000E82EFCD79E96C69E25C5C9FFFF0E9EB62D
:105FE00002D0E82EFCD79E96C69EC952FF0E9EB6E2
:105FF00002D0E82EFCD7898A0F01C950FF0AD8A425
:106000009BEF32F00501FE0E336FDDEC2AF0ABC5DD
:1060100034F5ACC535F5ADC536F5AEC537F5AFC50C
:1060200038F5B0C539F5B1C53AF50784B6C166F1A2
:10603000B7C167F1B8C168F1B9C169F14BC14FF19E
:106040004CC150F14DC151F14EC152F157C159F1FE
:1060500058C15AF1AEEC1DF000C13BF501C13CF551
:1060600002C13DF503C13EF505015D673FEF30F02C
:106070005E673FEF30F05F673FEF30F0606743EF00
:1060800030F050EF30F05DC504F15EC505F15FC53D
:1060900006F160C507F129EC28F003BF9BEF32F051
:1060A00059C13FF55AC140F5B5C541F5B6C542F5F0
:1060B000A1EC25F036C645F537C646F50101036B60
:1060C000026B1AC600F11BC601F101AF6CEF30F094
:1060D000FF0E026FFF0E036F0101076B066B1CC6FC
:1060E00004F11DC605F105AF7AEF30F0FF0E066F23
:1060F000FF0E076F2EEC28F00101076B066B1EC622
:1061000004F11FC605F105AF8AEF30F0FF0E066FF0
:10611000FF0E076F2EEC28F00101076B066B20C6FF
:1061200004F121C605F105AF9AEF30F0FF0E066FBE
:10613000FF0E076F2EEC28F0D890010103330233D5
:1061400001330033D89001010333023301330033AC
:1061500000C147F501C148F50101036B026B22C67E
:1061600000F123C601F101AFBAEF30F0FF0E026F6C
:10617000FF0E036F0101076B066B24C604F125C6F1
:1061800005F105AFC8EF30F0FF0E066FFF0E076F89
:106190002EEC28F00101076B066B26C604F127C61A
:1061A00005F105AFD8EF30F0FF0E066FFF0E076F59
:1061B0002EEC28F00101076B066B28C604F129C6F6
:1061C00005F105AFE8EF30F0FF0E066FFF0E076F29
:1061D0002EEC28F0D8900101033302330133003351
:1061E000D8900101033302330133003300C149F574
:1061F00001C14AF50101036B026B2AC600F12BC6EF
:1062000001F101AF08EF31F0FF0E026FFF0E036FD7
:106210000101076B066B2CC604F12DC605F105AF15
:1062200016EF31F0FF0E066FFF0E076F2EEC28F011
:106230000101076B066B2EC604F12FC605F105AFF1
:1062400026EF31F0FF0E066FFF0E076F2EEC28F0E1
:106250000101076B066B30C604F131C605F105AFCD
:1062600036EF31F0FF0E066FFF0E076F2EEC28F0B1
:10627000D89001010333023301330033D890010178
:10628000033302330133003300C14BF501C14CF538
:106290000101036B026B02C600F103C601F101AFFD
:1062A00056EF31F0FF0E026FFF0E036F0101076B17
:1062B000066B04C604F105C605F105AF64EF31F0C5
:1062C000FF0E066FFF0E076F2EEC28F00101076B23
:1062D000066B06C604F107C605F105AF74EF31F091
:1062E000FF0E066FFF0E076F2EEC28F00101076B03
:1062F000066B08C604F109C605F105AF84EF31F05D
:10630000FF0E066FFF0E076F2EEC28F0D8900101EC
:106310000333023301330033D890010103330233D6
:106320000133003300C14DF501C14EF50101036B8E
:10633000026B0AC600F10BC601F101AFA4EF31F008
:10634000FF0E026FFF0E036F0101076B066B0CC699
:1063500004F10DC605F105AFB2EF31F0FF0E066F87
:10636000FF0E076F2EEC28F00101076B066B0EC6BF
:1063700004F10FC605F105AFC2EF31F0FF0E066F55
:10638000FF0E076F2EEC28F00101076B066B10C69D
:1063900004F111C605F105AFD2EF31F0FF0E066F23
:1063A000FF0E076F2EEC28F0D89001010333023363
:1063B00001330033D890010103330233013300333A
:1063C00000C14FF501C150F50101036B026B12C60C
:1063D00000F113C601F101AFF2EF31F0FF0E026FD1
:1063E000FF0E036F0101076B066B14C604F115C69F
:1063F00005F105AF00EF32F0FF0E066FFF0E076FDD
:106400002EEC28F00101076B066B16C604F117C6C7
:1064100005F105AF10EF32F0FF0E066FFF0E076FAC
:106420002EEC28F00101076B066B18C604F119C6A3
:1064300005F105AF20EF32F0FF0E066FFF0E076F7C
:106440002EEC28F0D89001010333023301330033DE
:10645000D8900101033302330133003300C151F5F9
:1064600001C152F507940501200E326F899A400E42
:10647000C76E200EC66E9E96C69E060EC96EFF0E95
:106480009EB602D0E82EFCD7898A899A9E96C69E2F
:10649000020EC96EFF0E9EB602D0E82EFCD79E9665
:1064A000C69E27C5C9FFFF0E9EB602D0E82EFCD7B8
:1064B0009E96C69E26C5C9FFFF0E9EB602D0E82E48
:1064C000FCD79E96C69E25C5C9FFFF0E9EB602D07C
:1064D000E82EFCD725EE33F0322F02D07BEF32F0DE
:1064E0009E96C69EDECFC9FFFF0E9EB602D0E82E56
:1064F000FCD76CEF32F0898A899A9E96C69E050E6B
:10650000C96EFF0E9EB602D0E82EFCD79E96C69EA0
:10651000C952FF0E9EB602D0E82EFCD7C9B086EF56
:1065200032F0898A0501200E2527E86A2623E86AC9
:106530002723E86A2823120021C500F122C501F1B2
:1065400023C502F124C503F1899A400EC76E200EBF
:10655000C66E9E96C69E0B0EC96EFF0E9EB602D0EC
:10656000E82EFCD79E96C69E02C1C9FFFF0E9EB6BE
:1065700002D0E82EFCD79E96C69E01C1C9FFFF0E31
:106580009EB602D0E82EFCD79E96C69E00C1C9FFDB
:10659000FF0E9EB602D0E82EFCD79E96C69EC9522C
:1065A000FF0E9EB602D0E82EFCD725EE33F0050193
:1065B000200E326F9E96C69EC952FF0E9EB602D026
:1065C000E82EFCD7C9CFDEFF322FDAEF32F0898A0E
:1065D0001200899A400EC76E200EC66E9E96C69E09
:1065E000900EC96EFF0E9EB602D0E82EFCD79E9686
:1065F000C69E000EC96EFF0E9EB602D0E82EFCD7D6
:106600009E96C69E000EC96EFF0E9EB602D0E82E64
:10661000FCD79E96C69E000EC96EFF0E9EB602D097
:10662000E82EFCD79E96C69EC952FF0E9EB602D09B
:10663000E82EFCD7C9CF2DF59E96C69EC952FF0EF7
:106640009EB602D0E82EFCD7C9CF2EF5898A12005B
:1066500015EC27F0B5C5E8FFD70802E315EC27F0E5
:10666000B5C5E8FFC80802E315EC27F0B5C5E8FF9B
:10667000B90802E315EC27F0B5C5E8FFAA0802E364
:1066800015EC27F0B5C5E8FF9B0802E315EC27F0F1
:106690008DEC2BF0A3EC2FF0F29CF29E8B94C69A1B
:1066A000C290898C9482948C720ED36ED3A4FED740
:1066B00089968A909390FF0EE8CF00F0E82EFED7DF
:1066C000002EFCD78150F294F29A9E909D909E925B
:1066D0009D92F298F292F290F286F28E0300FF0001
:10BF0000E844F926000C160C2B0C3F0C520C640C68
:10BF1000760C860C960CA50CB30CC10CCF0CDC0C6B
:06BF2000E80CF40C000C1B
:00000001FF
